:020000040000FA
:20000000803F00320000000000000002DCBD0000000000C2AA32000000000002DC86000052
:2000200000000010990802DC42000302DDF502DC662A532D31302056455220322E303720B5
:200040002AC2AF7590FF75B0FF7581DF758961758DFF758BFF75CBFF75CAF475C83D7598B0
:200060005075870075885075B80175D000E47801F608B800FB7506FF7507FF750BFF750C71
:20008000FF75D0181278ED908080740FF01191800D758390E4F07583C0F4F56AF0227481ED
:2000A00090E007F0E490E006F090E000E4F0A3F07D007E007F007B097A101249B7EF2410FB
:2000C000FFDAF70FDBF27D031278DBDDFB75688075A080743831307A05313C743831307A45
:2000E000323142743831307A14314274383130740831301278ED740131301278ED740631F4
:20010000301278ED740C7800F208123AFB1278ED90FF9274407B08123B06123B1A90FE38B0
:20012000C3123AE0123B2790FE40C3123AE080157800F2087480F208B809FB221278EDDA7B
:20014000FB22DAFE221264F2E574F4A2E475F00092F0E575F423543E45F0F559B401061213
:200160006737126761E53390B000F0E559B43002415575686175A0619051DC78007900E4BF
:2001800093F20809A3B910F7B8800280079051DC790080EB75A0631201C01264DC75A062F0
:2001A0001201C075A0651201C075A0661201C075A0671201C01266C175A06C1201C080066F
:2001C000E4F8F2D8FD2275A0647568647881E2540FF2F5317882E2F5227806E2F523C21805
:2001E000753216D22FD22E7884E254F34404F290648012022A85F05A75828712022A85F030
:200200005B12022A85F05C752F07E55AB55B028030B55C02802BE55BB55C2675686475A03D
:2002200064788079871202388017780375F000E025F0F5F0A3D8F8227A03E3F20809DAFAF9
:200240002275686475A06478877980120238788A7980120238791090E008E9F0755A107509
:200260005B0090FFFFF090E404E4F0A3F0D55BF6D55AF309B930E0780090517F740BF090D5
:20028000F30075685075A050E893F208B800F979007A0090FA8075685175A0517800E8932F
:2002A000F30809B80CF80ABA04F2E475685175A051F309B97DFB7980F309B900FB43901F84
:2002C00012009190517F7408F07530FFE559B43002802CB41202802D906485E559F0B4016A
:2002E0000C90FF12123D00123B4F1278F690FECF123D00123B4FC299C29875A8FB800B75D1
:20030000A88102D1E0D270026D00209211303303020349D233301303125FBA0203492033C2
:2003200003020349C233301303125FBA75686375A06378017905E2547070037405F3E824C6
:2003400010F8E92410F9B881EDE510B511030203F375D01075686775A067E208F555E25424
:200360007FF55908F55675D018755300123E76301803020391758362851782E4F0058205B9
:2003800017E555F005820517E556F00517E52054C3C2AC75686675A06675D0087490253143
:2003A000B50A028003FAF309E555547FF309E55530E704E5598001E4F30975D018E555204F
:2003C000E72312460A303B1D75686675A06675D00874B02531B50A028004F50AF309747B75
:2003E000F309E4F30975D018302E04C22ED299D2AC8000E500B50103020B3B75686575A0CC
:2004000065A800E2F550050020E71CE5027003020B3B74022505F8E550F60505E505B4046F
:200420005875050302047954F0B4F02CE55020E31F301616540F700C7502F0750501750D5E
:2004400000020B3BB407030207F4120B46020B3BB4FE02D235020B3BB4A0028003B4D00688
:20046000120B46020B3BA802855002750501B8F005D2580207F4020B3BE502C4540775F04E
:2004800003A4900486730204A40204E80205350205410206640207580207640207B9120BF3
:2004A00046020B3BE502540FB531F3E505B403057505018003020B3B755301850355123EA9
:2004C00076207D1B2018187568628568A0A8177401F2080517E503F2080517E4F205170296
:2004E0000B3B120B46020B3BE502540FB531F3E505B403057505018003020B3BE50460B8FB
:20050000755301850355435580123E76207D1E20181B7568628568A0A8177401F208051733
:20052000E5034480F2080517E504F20517788AE504F6020B3B120B46020B3B120B46020BBE
:200540003BE502540FB531F3E505B403028003020B3B750501E503B40117301214E50470F1
:200560000BC226754B00754C00020B3BD226020B3BB4403230132CE504C39440501475830E
:200580006285178274FD7A03F005820517DAF9020B3B75836285178274FE7A03F00582055C
:2005A00017DAF9020B3BB4065230174CE5066003020B3BE507600EB401F6E504788BF612DB
:2005C0000B51020B3BE504C3940D500585044F8003754F0C7415C3954FF532E56D70061279
:2005E00078ED123BA1205904788480027886E6F55A08E6F55B1210C7020B3BB426173017D3
:2006000011E506700DE507B40108E504788CF6120B51020B3BB462097506FF7507FF020BFE
:200620003BB463097506FF7507FF020B3BB46506850406020B3BB46406850407020B3BC373
:20064000947B401720321420331175836285178274FF7A03F005820517DAF9020B3B120B37
:2006600046020B3BE502540FB531F3201106120B46020B3BE505B402028003020B3B750500
:200680000190F600E50323F5F093F55AA3E5F093F55BC05AC05B9063B0E525F0A3E570F0EC
:2006A000A3E571F0A3E572F07525007570FF7571FF7572FFD279E55B540FF550C205125BB7
:2006C00022D05BD05AE55A30E30280030207287570FF7571FF7572FF20E23AE55BC4540F49
:2006E000F550E55A54037029752500900742E55B540F23F5F093F55EE5F0A393F55F74703F
:20070000255EF890FA94E55F93F55FE6555FF68010F525800CE55A5403F525E55B540FF507
:2007200050D279D205125B229063B0E0F525A3E0F570A3E0F571A3E0F5725325FCD22E02EA
:200740000B3B00000001000200030103010402000201020202030204120B46020B3B120B68
:2007600046020B3BE502540FB531F3201406120B46020B3BE505B403F8750501E504700A6C
:20078000E503C394205003750320E50323F55D85045C755F00755E40126832855C5B855D1C
:2007A0005C126ADA126ADA7886E55AF67887E55BF6D2591210C7020B3B74CA250DF8E5031D
:2007C000F6750501050DE50DB4010878CAE6B4411D801EB4030878CBE6B531128013B404E4
:2007E0000878CCE6B410078008C394144003120B46020B3BE50DC394095003020B2574CA06
:20080000250DF874F7F6E50D7003020B2578CE7900E6B4F708E9547F600C020B2529F908DA
:20082000B8DFEE020B2578CDE6B411028009B412030208CE020B25E50DB40B028003020B70
:200840002508E670EF08E6B4081008E6C3941950E3E6F55312615E020B25B4095008E6C3EC
:20086000940450D0124DC3740FF554F555F556F5579063B0E0F5F0A330F005E0540FF55435
:2008800030F105E0540FF55530F205E0540FF55630F305E0540FF5577550127551007552D5
:2008A00009755300755F041260F0020B25C394045019E6F55208E6C39438500FE69063E96C
:2008C00093B4FF028005F553126217020B2508E670F908E6F552C3940450030209F5E6B472
:2008E0001002800302099008E67008C2051258E1020B2514600814603B14605780CD08E6ED
:200900006006146007020B25C2188012D218C234E56D7008742078BFF6123B4FD255A21870
:20092000B3E56A92E7F56A7583C0F0124A701266C1020B2512643D1278D312659DC27B128B
:20094000546112B816756D00D27B1254611265F4020B2508E6C39404502F90098CE6C0E0FC
:2009600093906485F01266C1126719C23478BFE6B453037420F6D0E0B4030BD234E56D70CF
:200980000878BF7453F6123B4F020B2500151615B408BD08E6C3941950B6E6B41102D251A0
:2009A000B41302D25190619A75F005A4F5F090619A7954E5F093A3F709B959F708E6C3951B
:2009C000588557F0A4F5F075686475A064A854E2A955B900028004031980F7F550E556F48E
:2009E0005250E55045F0A955B900028004231980F7F2020B2508E6C394384003020B25E6FF
:200A00009063E993B4FF03020B25F5537003020B0175F00614A4F5F09063477954E5F0933F
:200A2000A3F709B95AF7E552C423F55275686075A060E5546003020A7CE6B40C02D253B44D
:200A40000D02D25308E68559F0A4C39558F5F0E5522555F8E2A956B900028004031980F711
:200A6000C0E0E557F4F557D0E0555745F0A956B900028004231980F7F2020B25E50DC3946B
:200A80000D5003020B25124DC378D5E65403F55A18E6C4F55B18E6425B18E6C4F55C18E60B
:200AA000425CE554B40208755D00755E00801A78CFE69063B12582F582E023F5F09063395F
:200AC00093F55DE5F00493F55E755F00126892E5522555F8E2A956B900028004031980F736
:200AE00054FC455AA956B900028004231980F7E2E5522557F8E55BF208E55CF2D250020BED
:200B000025E50DC394115003020B2508906100E552C42582F582E6547FF0A308B8DAF712D0
:200B20003C76123B4F120B46305310C253C205D27B125461C205D27B125461E500B5010308
:200B4000020BA40203F3E4105804F502F505F50D22755A00788BE6F55B08E623F55C455B7D
:200B60007004749D8031126AEB755D00755E20755F001268A592795006126BD212693D8533
:200B80005B5D855C5E755F641269C07F0D126B99E55C307902F404906480F0906487F09006
:200BA000648AF022532EF0E52054C3B4C2028003020C39D273305105C2511266C190640E4D
:200BC000E0FFA3E0FEE5152404F51550050514531403E5122468F568F5A0A8137950E26076
:200BE00041A2E79270E4F208E2F7E4F20809B953F775686275A0627950A817E550E5512EB1
:200C0000F5518FF0E552A485F052435004E7F20809B953F9051705170517307005120CF6DA
:200C200080B0120CF685125C85135D85145E85155F12685050031266C1A29392D5203970DD
:200C400030D502807A9064007A04E0B41705A3DAF9800375437F906404E004F53ED2399097
:200C600064007A04301808301A02D219020CEF75686275A062E0B41702802BF55B7402A892
:200C800017F2080517E55BF2080517E4F20517087402A817F2080517435B80E55BF208052F
:200CA00017747FF20517A3DAC68044203841809530D5F8E53E7038C239301803020CEF90CC
:200CC00063017A0875686275A062E030E4190582E01582F55B7402A817F2080517E55BF2A0
:200CE000080517E4F20517E5822410F582DAD5A2D5B39238800EE5132404F5135005051207
:200D000053120322C2A98523F053F003906406E054FCF523E5F04223D2A9201803020E2698
:200D2000752F00E52054C3B4C202D27D906405E0C31390F980937880F61245AD124628303F
:200D40003A3275836275686375A0637801E230E617E4851782F00582051708E2547F18F033
:200D600005820517E4F00517E82410F8B481DED255020E2630555EC2557880E6F53FC21975
:200D8000124937F543124754906407E014FDE5232323540323900D99738006800F801C804E
:200DA000277541008D40855842020DD0E523C45403F5418D40855942020DD07541008D40E3
:200DC000855842C256020DD07541008D40855842201A53802F201903020E26C21975686293
:200DE00075A062A817E4F2080517E54175F00CA425422418547FF2080517E4F205171247B1
:200E0000541247A175686275A062A817E4F2080517E54175F00CA4254224184480F2080574
:200E200017E543F20517E516B517028078E517C3951675F00384E5F0600B1266C112671646
:200E40008517168049758362851682E0F47013051605160516A23292D5125FEDA2D5923224
:200E6000802C14700A051605160516D232801F14700B0516051605161260D08011E5160492
:200E8000F582E030E705123EC38003123F54E516B5179AE510B51107E500B5010580060259
:200EA00003490203F3E5287003020EC97A0090FA8CEA935528600DEA23C42413FF7E007D9C
:200EC000A01249B70AEAB408E553A8DD752F007533001210ACE550C3948040067401456B62
:200EE000F56B43A82253A8DD7533011210ACE550C394035005755000800AE550C394FE4039
:200F0000037550FF855045E56B54036003B40302E545E56B20E308755C0085485D800F75A9
:200F20005C00755D00755E0085485F126832E56B20E20B755E0085475F1268248009755E83
:200F40000085475F126832E56B20E10B755E0085465F1268248009755E0085465F12683291
:200F6000E56B20E00B755E0085455F1268248009755E0085455F126832855C5E855D5F12B9
:200F800068D91268D9855E58855F59854FF0E55E20E019E55FA485F05CF55D755E00E55012
:200FA000600205F085F05F126824801EE55FF404A4755C00755D0085F05EF55F126832056F
:200FC000F0755E0085F05F126832E55CB57E07E55DB57F028008855C49855D4AC2597884E6
:200FE000E558F67885E559F6855C7E855D7F301403125E6C854748854647854546754500BA
:20100000C3E56B33F56B43A82253A8DD7533021210ACE550C3954E5002F404F551C3940407
:201020005005202F02804BE55075F00DA4E5F0B54F05202F028025F54F7415C3954FF53285
:20104000202F1930170C755200854F5375540012604FE56D70061278ED123BA185504E20ED
:201060005904788480027886E6F55A08E6F55B1210C743A82253A8DD7533031210ACE550A8
:20108000C394C0500F202008D226301203125EF3D2208013302008C226301203125EF3C2C3
:2010A00020754B00754C0043A8228061C0A875A88990B000E5335403F533F0755050D55092
:2010C000FDE0F550D0A822854FF0E55A20E019E55BA485F05CF55D755E00E55B600205F0C7
:2010E00085F05F126824801EE55BF404A4755C00755D0085F05EF55F12683205F0755E00C6
:2011000085F05F126832855C49855D4A2275D01875686475A0647809E2047883F61245AD64
:20112000124628A23372327239B3823A5004C224801F20241CA23AB372395041754B007563
:201140004C00D224C225780CE27881F608E4F6802C2025297881E6F55C08E6F55D455C60A4
:201160001A755E00755F801268325006755C00755D00E55DF618E55CF68002D2252026063D
:2011800020250302120E75F000302605780AE2F5F0302509780BE225F0500274FF700302CA
:2011A0001208F5F0E535C3948020270440068023402C803AF404C333500114A4755C0075A8
:2011C0005D00755E0085F05F126832855D4C855C4B803BC333A485F04C754B008030F87413
:2011E0007FC398C333A485F04C754B008020C333A4755C00755D00755E0085F05F126832CA
:20120000855D4C855C4B8006754B00754C00305F0BC25F12643D1266C1126716305205129E
:201220005FEDC252305E0BC25E1264A61266C1126716C2A9E53A7012750A00750BFF750C26
:20124000FF301503126033753A0AE53B701D20370BA2359237C235303711800F20350A12CB
:2012600060D0125FEDC2378000C235D2A98000302D16E5387012C22DE56D6009436E80A2E6
:201280005B922D8003123B4F30314FE539704BE56AF4F56AE530C4540F903C6793F5F0C43F
:2012A000540FB4090478698002786AE5F0540F90FA8C93F5F056600A753908E5F0F456F674
:2012C0008007753920E5F046F6758390E569F0E56AF4F56A7583C0E56AF08000C205E56DB0
:2012E000B40403124D16124AB775500075686375A063E550C42401F8E25403F557E550233B
:20130000C44257E550C42403F8E2F55408E2F556E550C42408F8E2F55508E2F55808E2F599
:2013200059305005D273124E78E55554C06018788FE6F55F08E6F55EE557C4540FFF126A8C
:2013400051E55FA2E09272E55754F04401FF1250FD8D5A8E5BE55754F04402FF1250FD8DCE
:201360005C126AEB126AEB126B24758360E55554C0604C20724230E61CE559240EF582E083
:2013800003035403F55DE5592406F582E0F55EA3E0F55F801AE559240FF582E023235403B6
:2013A000F55DE559240AF582E0F55EA3E0F55F1268A54004C273806C125122D27380658536
:2013C0005A51855B52855C53758360E55520E51CE559240EF582E05403F55DE5592408F57A
:2013E00082E0F55EA3E0F55F785A801CE559240EF582E023235403F55AE5592404F582E083
:20140000F55BA3E0F55C785D1217501268A585515D85525E85535F1268A5400612680112AA
:201420004B4CC27375686375A063E550C4240CF8E2F55C08E2F55D455C604DE559241EF5D5
:2014400082758360E0F4C31390FA0093F55FE559241FF582758360E0F5F0755E00E55FC3A8
:20146000940A4012A4E5F075F004A4240A500205F085F05EF55F1268325006755C00755DB5
:2014800000E55DF218E55CF2124B5CE55754F02417FF1250FD8E5E0F1250FD8D5F1268CD6E
:2014A000E5286075E55090FA8C93F5F055286069E55E455F600302173AE5F0F45228758369
:2014C000637D05EDC42400F582E0540C700BDDF3D27F20050A7E3080087E70C27F80027E6B
:2014E00074E550C42400F582E0540FFCEE540FFDC4F582E0C39C500AE0045407307F02543F
:2015000003F00DEEC404540F8DF0B5F0028003ED80DEE550C4F582E4F0758363E550C42404
:2015200005F582E0858251540775F003A49015317302154902154C02157702159602165DD4
:201540000216A102154902154902173AE55754F02413FF1250FDEEB55E02800540030217C6
:201560003A758363E550C42405F5827402F0124CD220701102173AE55754F02413FF12509B
:20158000FDEEB55E0B7583638551827403F080032072F202173AE5562304F5F0E55924190C
:2015A000F582758360E0A4E5F0F552B55E0302163F92D5500E855E5C855F5D85525E755F01
:2015C00000800685525C755D00126832AC5CAD5DE5592415F582758360E0F582C3940F407F
:2015E00009F5F0A4E5F0240F8002E582F5F0A4755C00755D0085F05EF55F126832AE5CAFB0
:201600005D126CC1E55C455D6035855C5E855D5F8C5C8D5D126832E55C600590F800800505
:2016200090F700E55D9320D505FDAE528004F4FDAE52E55754F02413FF1249B702173A7552
:201640008363E550C42405F5827404F07D00AE52E55754F02413FF1249B702173AE55623AD
:2016600004F5F0E5592419F582758360E0A4E5F0F552FE7D00E55754F02413FF1249B7E56F
:2016800052C31392D57D00FEE55754F02417FF1249B7E4A2D592E7FD7E000F1249B70217EB
:2016A0003AE55E455F700302171BAC5EAD5FE5592416F582758360E0F582C3940F4009F50A
:2016C000F0A4E5F0240F8002E582F5F0A4755C00755D0085F05EF55F126832AE5CAF5D125E
:2016E0006CC1E55C455D6033855C5E855D5F8C5C8D5D126832E55C600590F800800590F70F
:2017000000E55D93855C5E855D5FF4FD7E00E55754F02413FF1249B702173A758363E5505A
:20172000C42401F582E0547FF01249797E007D00E55754F02413FF1249B7E55004B4080218
:20174000800CB40402D20505500212ECC25080167903758363E5575403232324E0F582E064
:20176000F608A3D9FA22E530540FB40F17E56D7013904003E020E10C12460A303B062033C6
:20178000030219C3C273D2791264F2126696202B03021E2C752F00790078C0E620E0110983
:2017A00003B905F808B8C703021E2CE6790080EC75F003E8C394C0239017BC73800C801F44
:2017C000803280458058806B807E9017D0E9A47302185D02186202186702186C021E2C9084
:2017E00017E5E9A473021E2C021E2C021E2C0218710218769017FAE9A47302187B0218801E
:2018000002188502188A02188F90180FE9A47302189F0218E202191D02194E021E2C9018DB
:2018200024E9A4730219B0021A3D021A96021B11021B8A901839E9A473021C8B021C9D0292
:201840001CD2021CFD021D0F90184EE9A473021D75021DAB021E2C021E2C021DE77550009A
:201860008030755001802B75500280267550038021755004801C755005801775500680124E
:20188000755007800D7550088008755009800375500A756D00C230C25B125B22021E2CE5C9
:2018A0006D7007E530540FB40F03021E2C12460A303B2C203329C221E5255403B40102D278
:2018C000215325FC12659DC27B125461127B5AC4540F42211265F4D27B1254617573FE0283
:2018E0001E2CE56D70F9C23478BFE6B453037420F6E576540370E8906485E4F01278EDC2AC
:2019000030123B1A90FF72C3123AE0123B2790FF7A12198A75540012199A021E2CE56D7072
:201920002AE576540370249064857415F01278EDC230123B1A90FF72C3123AE0123B279081
:20194000FF8212198A75540112199A021E2CE56D70F9C23478BFE6B453037420F6E5765465
:201960000370E89064857416F01278EDC230123B1A90FF72C3123AE0123B2790FF8A1219A1
:201980008A75540212199A021E2CC3123AE0753830D22D1266C112671922301612755012FA
:2019A000755100755210755303755F011260F022E56D700612460A203B03021A3A30330322
:2019C000021A3A12659DC27B1254617BFFE57020E0047B00801320E1047B11800C20E20495
:2019E0007B22800520E3027B33E5255403601D30E0115325FCEBB4FF05126EBE801C126EA2
:201A0000CB80175325FCEB126EDD800EEBB4FF05126ED08005126EDD8000906406E0532375
:201A20000154FE4223121E84B80F02800288301265F4124D16D27B125461021E2CE56D7035
:201A400052E530540FB40F02804912460A303B4320334012659DC27B125461752F0FC025DB
:201A6000C2051258E1D025E5255403600E30E0085325FC126EB380065325FC126EA8121E7F
:201A800084B80F02800288301265F4124D16D27B125461021E2CE56D6021B40416E5732066
:201AA000E006125D57021E2CE57420E106125D0F021E2C0560753C00021E2CE57420E32E18
:201AC000906485E0B4152720341220100F121EAAD23475540312199A7453800AC234755497
:201AE0000112199A742078BFF6124967800DE56D701CE5255403600830E005121E72800B27
:201B0000121E7D7431F65325FC0525123B4F021E2CE56D6021B40416E57320E006125D5732
:201B2000021E2CE57420E106125D0F021E2C1560753C00021E2CE57420E22B906485E0B42A
:201B4000152420341220100F121EAAD23475540312199A7453800AC23475540112199A74EC
:201B60002078BFF6800DE56D701DE5255403600830E105121E72800C121E7D7432F65325DE
:201B8000FC432502123B4F021E2CE530540FB40F03021C7AE57520E31B1267371278EDC2C0
:201BA00030123B1A90FF22C3123AE0123B2790FF2A021C4F20E439125FED75310075221C60
:201BC000906481121BE9758288121BE975828B121BE9C2301278ED123B1A90FF32C3123AAD
:201BE000E0123B2790FF3A8066E4F0A3741CF02220E024E4906480F0758287F075828AF07E
:201C0000C2301278ED123B1A90FF42C3123AE0123B2790FF4A8038E56D600DB4040280082E
:201C2000B406028003B40755200452C2051278ED1258E15325FC78B07420F608F6C230122E
:201C40003B1A90FEBFC3123AE0123B2790FEC7C3123AE0753830D22D301615755012755167
:201C600000755210755300755400755F011260F0E56D6006756D00123C76021E2C756D0039
:201C8000123C76123B4FC230021E2CE530540FB40F028006756D81756F00021E2CE53054E7
:201CA0000FB40F028029E52554036013B40108756D867561008015756D87756100800DE592
:201CC0006DB404028003756100756D84756F00021E2C12460A303B2220331F756D00E53096
:201CE000540FB40F02801312659DC27B1254611291B5D27B1254611265F4021E2CE5305485
:201D00000FB40F028006756D82756F00021E2CE530540FB40F028014E52554036008B40285
:201D20000E756D858003756D83756F00021E2C5325FC12460A303B3A203337E530540FB4E5
:201D40000F0280B6301618755012755100755210755302E4F554755F011260F01278D312CD
:201D6000659DC27B12546112B816D27B1254611265F4021E2CE56D600D7401121ECE056E0D
:201D8000436E80021E2CE57030E00C30E10D30E20E30E30F021E2C7400800A74018006743C
:201DA0000280027403123DC5021E2CE56D60137402121ECEE56EC2E76002156E436E80027B
:201DC0001E2CE57030E00C30E10D30E20E30E30F021E2C7400800A74018006740280027437
:201DE00003123DC5021E2CA218B218E56A92E7F56A7583C0F0301812C234E56D700874207F
:201E000078BFF6123B4FD2558000124A701266C1301619755012755100755210755301E4CD
:201E2000A21892E0F554755F011260F0788DE6F5F0603C08E67038E5F01423901E3F738008
:201E4000028010E57620E0217406F6056E436E80021E6FE57620E1117406F6E56EC2E76098
:201E600002156E436E80021E6F788DE4F608F6021EE5742078B0F608F65325FC22744678C3
:201E8000B0F608221264F278C07900E6600713400D09B905F9087900B8C3F0780F2275F0F2
:201EA00005E8A429901ED693F822124A7075530012465C30790675530112465CE52330E0AB
:201EC0000CC218E56AD2E7F56A7583C0F022788DF6087414F622000102030F0F0F0F0405FD
:201EE000060708090A532F00532EF0E56D536D7F30E7375325FCB4822C301805756E8680DC
:201F000027E52054C3B4C105756E8E801BB4C205756E918013B48105756E8B800BB4820508
:201F2000756E8C8003756E80D278E56E30E71CD279C230C25B756000E56DB40505756F0059
:201F40008003756F00753C00536E7F302D10E52F5403700AE5607006753C000228EFE56D00
:201F6000901F6A75F0035407A473021F82021F850220320224C702255A02254B022887023E
:201F800028870228EF30781090FB77123D00906480E0122D780228EFE53C700302202FE582
:201FA0003C123AD5C39402500302202F753C00207F17E567207708B46302807304801F7056
:201FC00005C277048018148015E56720770A600314800B04D2778006B46302805204F56771
:201FE000906480307702F404F565F0758287F075828AF01228F612292C123B4F3017309069
:202000006480E0123AD575F0A4A4755C40755D0085F05EF55F307F051268328003126824A3
:20202000855C53E55DC313F55475520112604F0228EFE56EC394164003756E15E56E90206B
:202040004675F003A4730220880220B10220DA02210302212C02214D02216E0221970221EF
:20206000B80221D90221FC02222102225002227F0222A00222CF0222F002231102234202C7
:20208000236B02239A0223C330791190FBEF123D0079091229641229800228EF75507F75DA
:2020A0005209123005207D0675530012615E0228EF30791190FBFB123D00790A1229641266
:2020C00029800228EF75507F75520A123005207D0675530112615E0228EF30791190FC073F
:2020E000123D00790B1229641229800228EF75507F75520B123005207D0675530212615EFF
:202100000228EF30791190FC13123D00790C1229641229800228EF75507F75520C123005A8
:20212000207D0675530312615E0228EF30790F90FCEB123D001233A01229C00228EF12348A
:2021400028207D0675530412615E0228EF30790F90FCBB123D0012319D1229C00228EF12AA
:2021600031C8207D0675530512615E0228EF30791190FC1F123D007905122964122980027E
:2021800028EF75507F755205123005207D0675530612615E0228EF30790F90FC2B123D00B8
:2021A00012298D1229C00228EF12302C207D0675530712615E0228EF30790F90FC37123DAF
:2021C000001229CC1229C00228EF123053207D0675530812615E0228EF30791190FC471253
:2021E0003D0079071229E1123B4F0228EF123085207D0675530912615E0228EF30791190E2
:20220000FC53123D0079081229E1123B4F0228EFD270123085207D0675530A12615E022855
:20222000EF30791590FC84123D007911D27B1229648D5A1229C00228EF75507F755211D233
:202240007B123005207D0675530B12615E0228EF30791590FC78123D007912D27B122964D4
:202260008D5A1229C00228EF75507F755212D27B123005207D0675530C12615E0228EF3021
:20228000790F90FCC7123D001231FB1229C00228EF123226207D0675530D12615E0228EFF6
:2022A00030791590FCD3123D007910D27B1229648D5A1229C00228EF75507F755210D27BDA
:2022C000123005207D0675530E12615E0228EF30790F90FCF7123D001233711229C00228EF
:2022E000EF1233CE207D0675530F12615E0228EF30790F90FCDF123D0012337E1229C00246
:2023000028EF123403207D0675531012615E0228EF30791590FC90123D00790DD27B1229C1
:20232000648D5A1229C00228EF75507F75520DD27B123005207D08D25175531112615E021E
:2023400028EF30791190FC9C123D00790E1229641229800228EF75507F75520E12300520BB
:202360007D0675531212615E0228EF30791290FDA8123D0090640FE0D271122D780228EFE1
:20238000D271123476207D0F90640FF01234CED25175531312615E0228EF30791190FC5FFE
:2023A000123D0079041229641229800228EF75507F755204123005207D0675531412615E38
:2023C0000228EF30791290FEF3123D00123B4F756F008526630228EFE56F70448563F0854D
:2023E000266320330C203211E560756000602E801A20F329756F01800620F221756F029000
:20240000FA9C123D00123B4F0224C4756F031239DD123B4F123A27906400E0F5670224C419
:20242000E56FB40368E560756000602C20E70B0561E561B4040D156180091561E561B4FF92
:20244000020561123B4F123A2775836474002561F582E0F5670224C475F000203393203275
:2024600098755067755117122FC3207D5775836474002561F582E567F01239DD123B4F12E4
:202480003A2774152561F55312615E8037E56FB4010A303311C270123A328028303207D2E2
:2024A00070123A32801E756F00436E8075531512615E75531612615E75531712615E7553A6
:2024C0001812615E0228EFE56EC394084003756E07E56E6002802130790F90FB86123D00AD
:2024E000122A8C123B4F0228EF12460A303B062033031230E20228EF307920E56E23902505
:2025000034F55A93F55BE55A0493855B83F582123D00122A631229C00228EF12460A303BD6
:202520001020330D123119207D07E5677003123A870228EFFB86FB94FBA1FBAEFBBBFBC8B2
:20254000FBD5FBE20403020105070630790612317E0228EF1231620228EF307803122BF093
:20256000E56E547F6008E5606004D27D805FE56EC394194003756E18E56E90258275F00303
:20258000A4730225CD02264A02266E0226970226C50226EE022712022733022754022775B4
:2025A0000227990227BD0227E102280502282902282902282902282902282902282902281E
:2025C000290228290228290228290228292079609063D0E0F5F0E560207D13253C25602505
:2025E000602560123AD530E241207F208005603A20E719E561B40302802AF909E5F013549D
:202600000FD9FB601F13056150FB8010E5616014F909E5F013D9FD33156150FB756000754C
:202620003C00800C756000753C00207D06307917307D05123D61800F90FD1B123D00122CC3
:2026400002123B4F122C6D0228EF30790F90FD26123D00122D551229C00228EF12345220FE
:202660007D098561527553011262170228EF30790C90FD32123D00122D6F0228EF123476E9
:20268000207D1178101234421234CE8561527553021262170228EF30791190FD99123D0093
:2026A0007811122D47122D780228EF123476207D1178111234421234CE8561527553031297
:2026C00062170228EF307912753D0390FD4C123D00122DBB1229C00228EFE53D12354720F2
:2026E0007D098561527553041262170228EF30790F90FD41123D00122D891229C00228EFFB
:202700001234EF207D098561527553051262170228EF307918753D0390FD58123D00122D4C
:20272000DD1237DD122E72123B4F0228EF12372F0228EF307918753D0390FD5D123D0012DD
:202740002DFD1237DD122E72123B4F0228EF1238BD0228EF307918753D0390FD62123D00EE
:20276000122E111237DD122E72123B4F0228EF12381A0228EF30791E90FD8F123D00123585
:20278000221237DD122E7212365A123B4F8561527553091262170228EF30791E90FD94125A
:2027A0003D001235361237DD122E7212365A123B4F85615275530A1262170228EF30790FE3
:2027C00090FD67123D00122F961229C00228EF1235CA207D0985615275530B126217022854
:2027E000EF30790F90FD03123D0012358A1229C00228EF1235DF207D0985615275530C1284
:2028000062170228EF30790F90FD0F123D001235AF1229C00228EF1235F4207D0985615260
:2028200075530D1262170228EF307933755CFD755DB475F00CE56EC3940EA485F05EF55FFB
:20284000126824855C83855D82123D00E56EC3940E90287C93F8122FB11229C00228EFE561
:202860006EC3940E90287C93F552123630207D09856152856E531262170228EF12131714E7
:20288000181519161D1E1F20792E9063D0E0B4030280028020E560601C20E70BE561B4026E
:2028A00002800F05618006E561600715617560008006756000307931C27490FD20123D003C
:2028C000E52054C0B48016E56D30E006D27474328004C274743178B4F608743AF6122C9B3B
:2028E000123B4F122D1F0228EF12324C0228EFC22F000002030A78BA30710108E567700480
:2029000074208009207704742B8002742DF6AF67126A87EFC4540F70047420800224300832
:20292000F608EF540F2430F6123B4F22E563B565047405802B2480F55AE5652480C3955A22
:2029400092D5123AD5F55AC3940A500B20D5047404800D7406800920D50474038002740776
:2029600078BFF622C27A7568648568A0E3FD207B02C313307C0478BC800278BB122AFB22B9
:20298000123B4FEDF563C313F565F567227568648568A07906E3FDC413135403F55A755C1A
:2029A000FA755DCD75F004A4755E00F55F126824855C83855D827A0478BB122BAADAFB2255
:2029C000123B4F8D63855A65855A67227568648568A07906E3FDC45403F55A243178BBF6AA
:2029E000227568648568A0E3F563F565F56778BB601DFF126A87EFC4540F600424308002F4
:202A00007420F608EF540F2430F6087420F62290FAA6122BAAB8BEFA227568648568A079E4
:202A200082E3FD20E00890FAE0755A00800690FAE4755A0178BA122BAAB8BEFA22E56F54DC
:202A40007F78B42431F622E56F2400758364F582E0FDFA123D4778B8122BAAB8BAFAE92416
:202A600030F622902544E56E1493F9E522FD0313D9FD4008755A0090FAAD8006755A0190FE
:202A8000FAAA790378BC122BAAD9FB22E531540FF56304F565F56778BD122B3022902ABF3D
:202AA00023F5F093F551E5F00493F552902ADDE5F093F9E5F00493FA85518385528222FB55
:202AC00040FB43FB46FB49FB40FB43FB46FB49FB4CFB4FFB52FB56FB59FB5CFB61000700B8
:202AE000070007000702030203020302030203020300040203020300050007FF126A87EE99
:202B000070067420D27A80022430F608EFC4540F7007307A04742080022430F608EF540F96
:202B20002430F62278B1536F7FE56F04122AFB22FF126A87EFC4540F600424308002742028
:202B4000F608EF540F2430F622536F7FE56F23755CF6755D00755E00F55F126824855C833F
:202B6000855D82E493F55AA3E493F55B2278B5E56620E30590FAA6802620E2165403700565
:202B800090FB6D801A30E00590FB6F801290FB71800D540320E00590FB75800390FB737923
:202BA00002122BAAD9FB7420F622E493F6A3082278B8E567540F2404F5F0C3940F4002F5E9
:202BC000F0E5F0122A9D122BAADAFB22E566540CB4081C78BCE567C4540F2404F5F0C394EB
:202BE0000F4002F5F0E5F0122A9D122BAADAFB22124DC375686378B079D0E2F30809B8B5ED
:202C0000F9229063D0E0F5F030F00A7582D1E0FA7BB4122C4430F1119063D2E0FAB4050406
:202C20007BB880027BB7122C4430F20A9063D3E0FA7BBA122C4430F30A9063D4E0FA7BBDA2
:202C4000122C4422EA902AC723F55193F550E5510493F551902AE5EA230493F5528550832F
:202C60008551828B18A952122BAAD9FB22758363E56124D1F582E0F5F02304902AE593FB5B
:202C8000E561B40109AAF0BA05047A08800974038561F0A42404FA123D1922E53030740171
:202CA000C4540F902D0C9370119063D0F078B6902D177908122BAAD9FB229063D0F075686D
:202CC0006075A06014701C207404781B8002785BE2FA123D477A0278B6122BAADAFBE9241A
:202CE00030F6227B00781AE2FA123D47EB75F004A424B5F87A02122BAADAFBE92430F60BCE
:202D0000BB03028006741A2BF880DC2200000000000000010101034E6F2053706C697490BF
:202D200063D0E070087A067B08123D19221470087A067B03123D1922E56175F004A42405EB
:202D4000FA7B03123D192275686075A060E561C42328F8E2227802122D47FDF55AFA123DD9
:202D60004778BB7A02122BAADAFBE92430F6227810122D47122D7822F563F565123AD5A2F0
:202D80007F9277F5671228F6227801122D47FD23235403F55A75F005A4755CFA755DB012A8
:202DA0002DAC78BA7A05122BAADAFB2285F05EF55F126824855C83855D82227801122D47FD
:202DC000FDC45403F55A75F003A4755CFA755DC4122DAC78BB7A03122BAADAFB22755004DD
:202DE000C27C122E2354C0232314F565122F65122DF3228565628566638567642275500897
:202E0000C27C122E23540314F565122F65122DF322755006C27C122E2303035403F565121D
:202E20002DF322A850122D47F566A85008122D47F567207C04780E8002780F122D47227846
:202E4000B47424F608E5652430F608E566C4122E62E566122E62E567C4122E62E567122EB0
:202E60006222540FC3940A400424418002243AF60822758363E56124D1F582E0F5F0902FD0
:202E80004493F55085655A85665B85675C126ADA126ADA126AFC755D0085505E755F001235
:202EA0006980855C58855D59855C5F755D64755E651269C0E55AC3940A78BB4007E55A1261
:202EC0002AFB807BE55A603D85585E85595F1268CD1268CD1268CD855E5F755D7B755E0047
:202EE0001269C0E55AFF126A87EE6005755A0A80CCEFC4540F2430F608742EF608EF540F84
:202F00002430F6803A742EF60885585E85595F1269DD1268CD1268CD855E5D855F5E755F59
:202F20009E1269C0FF126A87EE600678BB7F1080C0EFC4540F2430F608EF540F2430F674E8
:202F40002508F6222020202040408000204060004000E55AC55DF55AE55BC55EF55BE55C08
:202F6000C55FF55C22758363E56124D1F582E0902F4B93755A00F55B755C00126ADA126A6E
:202F8000DA122F521237EA2073051268A580031268921237F4227801122D47FD20E2087571
:202FA0005A0090FAAD8006755A0190FAAA1235A522122D47FDC313F55AC05A78BB122AFBBC
:202FC000D05A22C27DE53C123AD5C3307E0494088002940450028020753C00207F0DE5675E
:202FE000B55005753C008010056722E567B55105753C008003156722D27D22E563756864D5
:2030000075A064F222755100C27E122FC3207D1BE567207B0123F563A852122FFBE567126A
:20302000297375500A1230BD123B4F22755003755100D27E122FC3207D18E5675403030328
:2030400053633F1231E912299E75500A1230BD123B4F22755002755100D27E122FC3207D6C
:2030600023E567C45363CF4263E563A21892E0F5237806122FFBE5671229DB75500A12303A
:20308000BD123B4F2230700875500A7551018006755010755101D27E122FC3207D1EE567FA
:2030A000F563307004780880027807122FFBE5671229EE7550051230BD123B4F22E567C34C
:2030C0009565700474058012123AD5C39550927E9030DEE52F232354039378BFF622030466
:2030E0000706755010755101D27E122FC3207D28E56714F563F531906488F090648BF078DD
:2031000081122FFBE567122A977550051230BD123B4F1260A31260D022755001755100D297
:203120007E122FC3207D3A902544E56E1493F5F0E567600A90FA8CE5F0934263800890FA73
:2031400094E5F0935263E563F522906489F090648CF07882122FFBE567A2E0122A7212348A
:203160001E2275507F75510085675A856F67122FC385676F855A67207D0312317E2290FCB0
:20318000A8123D00122B24122B49855A66855B67122B6D122BB0122BCC123B4F22E523FD62
:2031A00003035403F55A755CFA755DF075F004A4755E00F55F126824855C83855D827A04BE
:2031C00078BB122BAADAFB22755001755100D27E122FC3207D12E567540323235363F312AB
:2031E00031E91231A612341E224263E563A21892E0F5237806122FFBE56722906413E0FD09
:203200005401F55A755CFA755DE875F004A4755E00F55F126824855C83855D827A0478BB3A
:20322000122BAADAFB22755001755100D27E122FC3207D17E56754015363FE4263E563904A
:203240006413F0540112320412341E229063D0E0606EF5F01232C1E2F70809DAFAE5F0B442
:20326000033EE56170128566501550755118755B651232D4704A803C1470148567501550CB
:203280008565510551755B661232D4703380257550678566510551D2711232D470228014C8
:2032A000756518756767755067755118755B661232D4700C1232F5122C9B123B4F122D1FF9
:2032C00022741A3074022440F87568608568A079657A0322A95BD27E20710585675A8767D7
:2032E000122FC3207107A95BA767855A67207D02E42274FF22E530307401C4540F90332ECE
:20330000933074022323F5F07568608568A030F004E412333930F105742012333930F2059A
:20332000744012333930F305746012333922010101010101010303030FC0E0241AF87965EC
:203340007A03E7F20809DAFAD0E0C403C0E0F552755319126217D0E0C0E0F55275531A12DD
:203360006217D0E0C0E0F55275531B126217D0E022123395C4235401F55A12338B22123361
:203380009503035401F55A12338B22755CFA755DFC1233B2227568648568A07913E3FD22EE
:2033A000123395135401F55A755CFB755D041233B22275F004A4755E00F55F126824855C0E
:2033C00083855D827A0478BB122BAADAFB221233E9207D14E5675401C4035363F71233F549
:2033E000E56712337A12341E22755001755100D27E122FC3224263E5637813756864856894
:20340000A0F2221233E9207D14E567540123235363FB1233F5E56712338712341E227550E4
:203420000A1230BD123B4F221233E9207D13E5675401235363FD1233F5E5671233A81234B7
:203440001E2275686075A060E561C42328F8E563F222755067755118D27E122FC3207D15C1
:20346000E567F5637802123442122D5D7550051230BD123B4F22E53C605130710575500C3A
:203480008003755032E53C123AD5C39402403C753C00207F17E567207708B55002802C0492
:2034A000801F7005C277048018148015E56720770A600314800B04D2778006B55002800B26
:2034C00004F567307702F404F56322D27D22E563123AD5A27F9277F5671228F6E565C5636F
:2034E000F56512292CE565C563F565123B4F22755002755100D27E122FC3207D24C205C256
:203500007B125461E567030353633F123580122D9575500A1230BD123B4FC205D27B1254A3
:20352000612275500CD27C122E23C4540314F562F565122F652275500AD27C122E23232318
:203540005403F562F56522755002755100D27E122FC3207D2AC205C27B125461E567C4536B
:2035600063CF123580122DC675500A1230BD123B4FC205D27B125461C205D27B125461220B
:2035800042637801123442E567227801122D47FD20E308755A0090FAAD8006755A0190FA2A
:2035A000AA1235A52278BB7A03122BAADAFB227801122D47FD20E108755A0090FAAD800634
:2035C000755A0190FAAA1235A522123609207D0E12361592E212361C122F9C123626221229
:2035E0003609207D0E12361592E312361C12359012362622123609207D0E12361592E11266
:20360000361C1235B512362622755001755100D27E122FC322E567A2E0E56322F5637801C1
:20362000123442E5632275500A1230BD123B4F2275507F755100122FC3207D1DE567D333F2
:20364000F563E563A852123442E56778BB122AFB75500A1230BD123B4F2278BF742AF62219
:203660009063C0785A7903123694D9FB229063C3785D7903123694D9FB229063C0785A79A0
:203680000312369AD9FB229063C3785D790312369AD9FB22E6F008058222E0F60805822262
:2036A000C27DE53C123AD56038146035753C001237EA755D009036E4F5F0C3940F400375E5
:2036C000F00EE5F023F5F093F55EE5F00493F55F207F071268921237F4221268A51237F4FC
:2036E00022D27D2200010001000200040006000A001200200038006000B001310203035D0E
:2037000005A89063C678627906123694D9FB229063C67862790612369AD9FB22E55DC55ACD
:20372000F55DE55EC55BF55EE55FC55CF55F22C273E53D60030237BF753D031236A0207DBA
:203740007ED250123702E56530E70E12370F7565007566007567008023122DFD1237EA1202
:203760002E111237FE1268A512366012370F1237FE1268A5500612367A1237F4123702D2CC
:2037800073122F657804E5661238087805E567123808780E122D47232354FC456504030386
:2037A000780E12380812370F1237DD122E7212398D123B4FD2738561527553061262172295
:2037C000126C81785AE6700774F0F608B85FF678B4795AE72430F60809B960F722E5732061
:2037E000E104122E3F221237C02285655A85665B85675C22855A65855B66855C6722856546
:203800005D85665E85675F22C0E075686075A060E561C42328F8D0E0F222E53D6003023873
:20382000BC753D031236A0307D030238BC123702E56530E70E12370F7565007566007567E6
:2038400004803AE565700DE5667009E567C39404500280EA122DFD1237EA123660122DDD89
:203860001237FE12367A1268A512366012370F1237FE1268A5500612367A1237F41237021A
:203880007806E5661238087807E567123808780E122D47C4232354FC45650303C4780E127E
:2038A000380812370F1237DD122E7212398D123B4FD25085615275530812621722E53D60CB
:2038C0000302398C753D031236A0307D0302398C123702E56530E71A122DDD1237EA122EB5
:2038E000111237FE12366D12689212370F1237F4805B758363E56124D1F582E0902F4493BC
:20390000755A00F55B755C00126ADA126ADA12695C12366012370F1237FE1268A550081264
:20392000367A1237F48026122DDD1237EA122E111237FE12366D12689212366012370F123A
:2039400037FE1268A5400612367A1237F4123702D273122F657808E5661238087809E567AE
:20396000123808780E122D4754FC456504780E12380812370F1237DD122E7212398D123BBE
:203980004FD25085615275530712621722C27F85655A85665B85675C85625D85635E85647C
:2039A0005F1268B950047405802F1268A55008126BD212693DD27F755D00755E01755F00B0
:2039C0001268A5400B207F047403800D74078009207F0474048002740678BFF62279B074CF
:2039E00020F709B9C0FB9064007850E0F608A3B854F9785079B0E6B4170E7420F709742D0C
:203A0000F7097420F7098019FA8954123D478955A954E493F709A3E493F709E5552430F71B
:203A2000090908B854D022E5612323FA7B03123D192290640078047417F0A3D8FC207004EA
:203A400079928002799C7F18E76023F5F0E5F013F5F050127A04906400E0B41704EFF0802F
:203A600005A3DAF580180FEF540770E18004EF2408FF09207005B99CCF8003B9A6CA123936
:203A8000DD123B4FC23022E56E149025449323903A9373800E800D800C80138023803380A3
:203AA0003280312222C226754B00754C002275836285178274FD7A03F005820517DAF92266
:203AC000305908C259754900754A007886E4F608F62222222220E703C27F22D27FF4042287
:203AE00092D575688075A080E420D503938001E0A3B40D0122F208B809EE227480B8090195
:203B000022F20880F8227800F2C0E008C3123AE01278EDD0E02408DBED2275688075A080BF
:203B200074807800F208221278ED74C07800F208221278ED74017800F208123AFB1278EDA2
:203B4000227800EA2480F208EBF208123AFB221278ED79B0123B1A123B5D123B27E709F2EE
:203B600008B809F92275688075A080740C7800F208123AFB1278ED123B1A90FAA6C3123A19
:203B8000E0906100EFC42482F582D3123AE0123B27D3123AE0B8090122C390FA9C123AE019
:203BA00022123B1A90FD7FC3123AE0123B27C3123AE01278EDE54F1268E5F5F054F0C460C7
:203BC000052430FB80027B207A41123B411278EDE5F0540F2430FB7A42123B411278EDE587
:203BE000321268E5F5F054F0C460052430FB80027B207A45123B411278EDE5F0540F243026
:203C0000FB7A46123B41753850D22D22E530540FB40F0122756900436A7FC205903C67E5F6
:203C200030300501C4540F93F5F090FA8C540F93C5F054F0F583B4900FE56945F0F569F0DE
:203C40007583C0E56AF0800FE56AF445F0F4F56AF0758390E569F030070A200607200504C6
:203C6000D20580B8C2052290919293C0C1C2C3C4C5C690919293E530540FB40F0790FECFCC
:203C8000123D0022E56D6003023CF478B07420F608B8C0FB20071275836175820078B3E00B
:203CA000F6058208B8BCF8802B200618E5205403700590FE88801A30E00590FE9380129051
:203CC000FE9E800DE52030E00590FEA9800390FEB4123CF530340578BF7453F6E5255403A4
:203CE0006012744678B0F630E006743108F68004743208F62278B3E493F6A308B8BEF822A4
:203D0000742078B0F608B8C0FB78B0E493B40D028006F6A308B8C0F32279C7E4F709F7093C
:203D2000EAC394084004244080022408F7906190EA24B0F8E6F008A3DBFAE582B4A0028023
:203D400003740DF0D2302279FEEAC3940C0950FB240CC333337583FB240C50020583F582E6
:203D60002290FEE9123D0075836374D12561F582E0FA75F003A4755CFB755D4085F05EF532
:203D80005F126824855C83855D8278BA7903BA060109E493F6A308D9F9123B4F753828D2B9
:203DA0002D22A230925BC2301278ED123B1A90FF52C3123AE0123B2790FF5AC3123AE07594
:203DC0003830D22D22C2D5C0E0903DD175F005A473300811801130090C800C300A07800791
:203DE000300B028002D2D5D0E07583605403C4232480F582E0540FF5F075686375A06378A4
:203E0000B090FF62E493F2A308B8C0F830D50790FB687A058019903E55E5F02393F8E5F0EB
:203E2000230493F9903E6BE5F093FA8883898278B8E493F208A3DAF91278ED123B1A906336
:203E4000B0D3123AE0123B279063B8D3123AE0753840D22D22FB40FB43FB46FB49FB4CFB47
:203E60004FFB52FB56FB59FB5CFB610303030303030403030507C27DE5535403B40201227F
:203E8000700478928002789CE555547FC394185003D27D22F5F094504003D27D22E5F0C3B9
:203EA000940840030880F82408F5F0E55530E70AE5F090FA8C9346F68008E5F090FA94936F
:203EC00056F6227583627853123F4C7855123F4C7856123F4C532FF8E52054C3B4C20BD2F4
:203EE00072E55330E204D2058002C2059063B0E556F0123FBEE55320E3511268011249792A
:203F000012510EC273124E78C273124B5C124C6B124998200519E52054C3B4C21285535A65
:203F200085555B435B809063B0E0F55C1246D1300719100516207213E52054C3B48202803D
:203F40000AD2059063B0E0F55680A722851682E00516F6227583627853123F4C7855123F59
:203F60004C0516532FF8E52054C3B4C20BD272E55330E204D2058002C205124433E5532030
:203F8000E30C124B4C20050630340312465C200516E52054C3B4C20F85535A85555B535B52
:203FA0007F755C001246D130071310051020720DE52054C3B482028004D20580BD22532FEA
:203FC0003F755700E530200704C205802BE52054C3B48219C20553567F906412E0C3955636
:203FE0005007E530C4D205800FE530800BD27FE530300504200601C4540F75F003A49040C2
:20400000027302402F02402F02402F02402F02402F02402F02403B02404102404102406C54
:204020000240850240AF0240AF0240AF0240AF3005062006037557020240A47557000240CF
:20404000A4758360300506200603755702741B3005052006022440F582E0F5F0E555547F94
:20406000C3C5F095F0500205570240A475836075821BE0F5F0E555547FC3C5F095F0500224
:2040800005570240A475836075821AE0F5F0E555547FC3C5F095F040030240A40557A3E599
:2040A00082B41DE7755860E55723C4F5598036858358858259741A2582F5821240CC85590A
:2040C00082E557C4232582F5590240E5E493F5F0E555547FC3C5F095F04001220557A3E572
:2040E00082B41DE822E52054C3B4814B300548906411E0F5F0E556C395F05003E48060C323
:20410000747F95F0700104755A00755B00755C7F755DFF755E00F55F126980E556B47F045E
:20412000747F803BC395F004F55F855D5E855C5D1269C0E55B8028E556547FC39440500497
:20414000D27EF404F5F0758360741D2559F582E0A405F07440207E0425F08003C395F09015
:20416000F90093C313F55675686375A0633034030242C9207F047E7080092005047E3080F5
:20418000027E747CFFEE540FFDC404F8E25470700E18E2540FF5F0C39C5004AB1DACF00D18
:2041A000EEC404540F8DF0B5F0028003ED80DABCFF31906485E0B41502800443530822EEB6
:2041C000540FFDC4F8E2540F7004AB1D80150DEEC404540F8DF0B5F0028003ED80E5126517
:2041E0000F80DC906485E0B4164490FA94EB935228EE540FFDC42402F8E2F5F0E555C2E7FD
:20420000B5F01EEDB51B028018C42401F8E25470700F90FA8CED934228EDC42405F8740533
:20422000F2EEC4540FB51D0280040DED80C7EBC42354F0425775F010EBA4F8E2540FFCEE04
:20424000540FFDC4F8E2C39C400AE2145407307F025403F20DEEC404540F8DF0B5F00280A2
:2042600003ED80DFEBC4F8207F04740780027403F202435B75686375A063207F07540712D4
:204280004295802B540320050512429580212404124295801AEBC4234257EB145403C4F968
:2042A0002401F8E2548FF2E92405F87400F222E5568543F0A485F05CF55D755E00755F1027
:2042C000126824855C5602435B207F057B0002435B2005057B0002435B7B04435780024387
:2042E0005BE55354F0F5F07B00EBC42402F8E2F9E555C2E7B5190BEBC4F8E254F0B5F002AF
:20430000802D0BBB08E37CFF7900E9C404F8E25470700E18E2540FF5F0C39C5004ACF0AB42
:204320001909B908E5BCFF07E553D2E3F55322EBC4F8E2540FFC7900E9C4F8E2540FC39CF2
:20434000400FE2C0E054F0F5F0D0E014540745F0F209B908E3EBC4F87407F2EBC404F8E5CC
:20436000535403600814600AE4D2E48008E4D2E68003E4D2E5D2E7F5F0E254F042F0E5579F
:20438000540345F0F208E555C2E7F28558838559820582124AAFFC20E206E555C2E7801AEF
:2043A00030040D855883E5592402F582E493800A758360E5592402F582E0F5F0E555C2E7A5
:2043C000F554EC30E006E5F0240CF5F0E554C395F0F554401C8CF020F3047C158002AC32FE
:2043E0000C9C400DE554C3940CF554C320E70280F008E554F208E556F2087400F2080808B9
:20440000855883E55904F582124AAFF208E558F208E559F2089063B0E0F208855883E559F4
:20442000241FF582E0C423F5F0541FF208E5F054E0F222C27F30070BE52054C3B482028035
:2044400002D27F75686375A0635353F7E553540360071460087FEF80067FBF80027FDF3000
:2044600003030244EA303403024527207F047E7080092005047E3080027E74EE540FFBEB95
:20448000C42402F8E2B5553018E2F5F0EFF455F06026E5F05FF2800818E25FF2547070184C
:2044A00020180620332020321D18E25407FC43538012455F12457E22EEC4540FB51B04439C
:2044C0005308220B80B943530480ED207F047E70800C2005047E3080052404FB7E74EBC4D7
:2044E00004F8E2548FF212455F227B00E55354F0F5F0EBC42402F8E2B555221818E2B5F0C3
:204500001C08E2548FF220331920321618E25407FC43538012455F7E7012457E220BBB081C
:20452000D12243530480F6207F047B0080092005047B0080027B04EBC42402F8E2B555165D
:2045400018E25FF220331320321018E25407FC43538012455F224353082243530480F7EB4D
:20456000C4F808E25407F5F0EBC42354F045F0F557755860E5575403C4C333F55922EE24C2
:2045800010FE540FF9E9C4F8E25407F5F0C39C4006E5F0145407F209EEC4540FB519E6EB52
:2045A000C4F8207F04740780027403F222789279A67A0AE6203305203202800147F7080905
:2045C000DAF1789C79A67A0AE647F70809DAF9303919906400E0B417028009301803201A20
:2045E000031245EC0582E582B404EA22C083C08278A6C39418C3940840030880F8240890D3
:20460000FA8C9346F6D082D083227892E66003C23B2208B89CF6D23B22789CE66003C23C30
:204620002208B8A6F6D23C2278A6E66003C23A2208B8B0F6D23A22EF20E704789C800278AB
:204640009275F008EE547FC394248428F8E6ABF0BB000280041B0380F792E022532FF9E530
:2046600053540F7004789B800A146003D27922D27A78A579677A0AE66002800B18E9C39497
:2046800008F9DAF3D279227A0820E7042319DAF9758362307A05788AE6801A851782158203
:2046A0007A0AE582C39403F582E07002800330E704DAEF7440F556851782E5535403F005E4
:2046C000820517E94480F005820517E556F0051722C068C01874682514F568F5A0A815E2ED
:2046E000602C74042515F51550170514531403E514B5120DE515B513081266C112671680A9
:204700001C74FFF274682514F568F5A0A815747FF208E55AF208E55BF208E55CF2D018D009
:20472000688568A022E55330E203C2F722300707E52054C3B48204790880027904756863E6
:2047400075A063780175F080E255F0F5F0E82410F8D9F52275686C75A06C78A679007A0098
:20476000D278E6602613F5F0E4500DAA194480307806C27844408958F309E954077008E5D9
:20478000F008B8B0DD800EE5F080DAE4F309E9540770F880ECEA6008A91AE344208959F3F6
:2047A00022C254906407E0FE1E75686C75A06CE5232323540375F003A49047BD730247C936
:2047C00002480302483A0248B3E540600515400248FA8E40A842E220E51208E2600588421E
:2047E0000248FAB84FF48558420248FA0541E523C45403F5F0C39541500375410085584208
:204800000248FAE540600515400248FA8E40A842E220E61218E2600588420248FAB800F466
:204820008559420248FA1541E54130E707E523C45403F5418559420248FA205640E5406082
:204840000515400248FA8E40A842E220E51208E2600588420248FAB84FF48558420248FA4E
:204860000541E523C45403F5F0C395415009D2561541205402800F8558420248FAE540608D
:204880000515400248FA8E40A842E220E61018E2600488428064B800F5855942805C1541BF
:2048A000E54130E709C256D25475410080988559428047E54060041540803F8E40E523C488
:2048C000540360131470071249235401800912492375F00384E5F0F541124923253554077F
:2048E000F5F0A842E26006E5F0600C15F008E8C394504001F880ED851842906408E0B40AA5
:2049000002801590491993F55F85435D85445E1269C0855A43855B4422305080C0D0E0F0D8
:20492000F5F9FD75F011E5342536A4F5F0758362853482E025F02212460A203B1675686756
:2049400075A067A81018790AE270191818D9F974408011124619203C09788AE670067440EE
:204960008002747F547F22789C790AE4F608D9FC78A6790AF608D9FC2290FA94E557C45477
:204980000F10E30A93552CF52C90E000F02293552DF52D90E001F02290FA8CE557C4540F21
:2049A00010E30A93452CF52C90E000F02293452DF52D90E001F0227583E88F82F000009038
:2049C000E002EEF0A3EDF02275686375A063E5595403F5F07408A42488F87A04E55930E6AD
:2049E00042124A5D124A53E090E000E030E0FC90E004E0F2A308E0F208124A53F090E000F7
:204A0000E020E1FC90E004E4F0A3F0DA0122E55920E70812695C2078C880C912693D2078C4
:204A2000C080C1124A5D124A53F090E000E020E1FC90E004E2F0A308E208F0DA0122E559CA
:204A400020E70812695C2078DA80DB12693D2078D280D3E55B44F0F583855C8222E55A542A
:204A600003C4F5F0E55BC4540F45F090E008F0227D817E007F137910C2AA1249B7EF24102C
:204A8000FFD9F779089063057405F0E5822410F582D9F51278ED1278ED7583637900E9C416
:204AA0002401F582E0540FF009B908F2D2AA22200402E022E49322906480E0755C00755D15
:204AC00000124AEEAC5CAD5D75686075A06090638078107A048C5C8D5DE2124AEEE55CF020
:204AE0000582E55DF00582E82420F8DAE822855C51855D52755D02755E94123AD5F55F1246
:204B000069C0755E00855B5F85515C85525D207F05126824800312683222EA2464C333FAFF
:204B200090F50093F55DEA0493F55E8B5F1269C0855A5E855B5F1269F5EA90F40093F55CD4
:204B4000EA0490F40093F55D12682422E55754F0032405F5827583637405F02285545C758B
:204B60005D00307311758360E5575403C4232411F582E0124AEE758363E557540F232480BB
:204B8000F582E0F55EA3E0F55F126824E52054C3B4C10C300509906413E030E202803175FA
:204BA0008363E5570354702408F582E0FC30E32085495E906413E020E105854A5F800EE5A0
:204BC0005E30E706E54A6002055E755F00126824E52054C3B4C10A300507906413E020E333
:204BE00016758363E557035470240CF582E0F55EA3E0F55F126832EC30E109854B5E854CDF
:204C00005F126824E52054C3B4C13B906410E0F55F906413E030E020E557035470240BF951
:204C20007568638568A0E3D333F5F0A4E5F004855FF0A405F085F05F755E002005051268A4
:204C4000328003126824AA5CAB5D124B1AE55C700DE55DC39460500674FFF55CF55DAD5C50
:204C6000AE5DE55754F0FF1249B72275686375A063E55754F003F5512405F87401F2758375
:204C800060E5592417F582E0F5F0E5562304A4AEF0E5592413F582E0FD124CA7E55754F00D
:204CA0002413FF1249B722ED75F0F0A4741025F0FDE5592412F582E0FB75F0FBA4E55623E6
:204CC00004F4A4E5F0F48DF0A4E5F0C313700104FD22C27075686375A063758360E559246B
:204CE00017F582E0FAA3E0F5F0C39A7003D2702292D5E5562304A4AEF0E5592414F582E0D8
:204D0000FD124CA7ED30D503F404FDE55754F02413FF1249B722124DC375686075A0609059
:204D200063B0E0F5F030F006755000124D4A30F106755001124D4A30F206755002124D4AD9
:204D400030F306755003124D4A22E55023C404F8E2F55154C0600122758363E55024B1F566
:204D600082E0F55225E02552F552E55120E505904D998003904DAE795AE55293F70905520F
:204D8000B95DF6758363E550232324E0F582795AE709F00582B95DF822017FFF01FFFF02CC
:204DA0007FFF02FFFF01FFFF02FFFF02FFFF0100000180000200000280000100000200006D
:204DC0000100009063B57850E6F008A3B856F9E530540FF5F0C39407400D23904DDF738000
:204DE0000E80178020802975500185F05180327550037551007552018027755003755102FA
:204E0000755203801C755003755104755205804E75500F7551007552017553027554038088
:204E20003D30073A200637E530C4540FF5F0C39406400F23904E38738024800E8017801E87
:204E4000801C43500485F053801443500C755300755401800943500C75530275540378500C
:204E60009063B0E6F0080582B855F89063B57850E0F608A3B856F92275686075A0602073C6
:204E800007A85908E2FC8002AC559063F0EC30E503024F5C54C07003024F1930E635E55993
:204EA000240EF8E2F5F05403F0A3E5592408125088A31250C430730302501CA3E5F012500C
:204EC000A49063F01250901250B79063F612509A02501CE559240FF8E2F5F0C45403F0A30F
:204EE000E559240C125088A3E5F023235403F0A3E559240A12508830730302501CA3E55967
:204F0000240EF8E21250A49063F01250901250B79063F612509A02501C531CEF758363E5A0
:204F2000575403232324E0F582785AE0F6A308B85DF99063F012509AE4F0A3E4F0A374045C
:204F4000F030730302501CE559240EF8E21250A41250B79063F612509A02501C54C070030A
:204F6000024FDD30E6271250D41250A49063F31250C49063F31250901268929063F0125055
:204F80009A30730302501C1250DD02501C1250D41250A49063F3E5F003035403F0A3E55991
:204FA000240A1250889063F31250901268929063F012509A30730302501CE559240FF8E2B7
:204FC000C45403F55AE559240CF8E2F55B08E2F55C1250B79063F612509A02501C758363CD
:204FE000E5575403232324E0F582785DE0F6A308B860F99063F3E4F0A3F0A37404F0755ACF
:2050000000755B00755C041268929063F012509A30730302501C1250DD02501CEC543023AC
:2050200023FB9063F0E02323421B7582F3E0C4421BAE1BE55754F04404FF1249B79063F17B
:20504000E0A3FDE0FEE55754F04406FF1249B79063F4E0A3FDE0FEE55754F04405FF1249AF
:20506000B72073239063F6E0A3FDE0FEE55754F04401FF1249B79063F8E0FD7E00E55754D0
:20508000F04402FF1249B722F8E208F0A3E2F022785AE0F6A308B85DF922785AE6F008A368
:2050A000B85DF92223235403F55DE5592404F8E2F55E08E2F55F221268A5126AFC126ADAF1
:2050C000126ADA22E5F003035403F0A3E559240612508822E559240EF8E2F5F022E559246C
:2050E0000EF8E25403F55AE5592408F8E2F55B08E2F55C1250B79063F612509A227583E853
:205100008F82E0000090E002E0FEA3E0FD2290FA94E557C4540F788F30E3010854079356C4
:20512000F62290FA8CE557C4540F788F30E3010854079346F62275686175A0617840906112
:2051400000E5595403C4F582E559543028F87910E55920E707E2F008A3D9FA22E0F208A3D9
:20516000D9FA2275686075A0607880906000E55923C45460F582E55923546028F87920E59D
:205180005920E707E2F008A3D9FA2288F0740E28FAF8E25430C5F0F8E0F208A3D9FAEAF8DD
:2051A000E254CF45F0F22275686075A0607910A859E493F2A308D9F99051EB7910E493F2C1
:2051C000A308D9F975686175A0619051DCE559C313F87910E493F208A3D9F9225F5F5F5FC8
:2051E0005F5F5F5F5F0D0000000000000000FFFFFFFFFFFFFF2F3B47FFFF00000E3C0000D5
:205200000000047FFF00047FFF4110110E3C0080000004FFFF0004FFFF4110220E3C00009D
:205220000000047FFF00047FFF8220330E3C0080000004FFFF0004FFFF8220040E3C0000D7
:20524000000004FFFF0004FFFF4110250E3C0000000004FFFF0004FFFF8220060E3C000094
:20526000000004FFFF0004FFFF4220070E3000000000047FFF00047FFF4110170E48008041
:20528000000004FFFF0004FFFF4110280E3000000000047FFF00047FFF8220380E4800809F
:2052A000000004FFFF0004FFFF8220090E300000000004FFFF0004FFFF4110290E4800002D
:2052C000000004FFFF0004FFFF82200A0E2800000000047FFF00047FFF41101A0E340080B7
:2052E000000004FFFF0004FFFF41102A0E4000000000047FFF00047FFF82203A0E4C008027
:20530000000004FFFF0004FFFF8220C27FE530300709300506200603D27FC4540F9053256D
:2053200075F003A47302534602534D02535402535B02536202536902537002537702538479
:2053400002539102539E9051FB1253B72290520B1253B72290521B1253B72290522B125382
:20536000B72290523B1253B72290524B1253B72290525B1254092290526B1253B790527BFA
:205380001253E02290528B1253B790529B1253E0229052AB1254099052BB12541F22905217
:2053A000CB1254099052DB12541F9052EB1254359052FB12544B22858357858258207F10EC
:2053C00030780C7559008557838558821251A722307A0C7559408557838558821251A722B3
:2053E000858357858258207F1030790C7559208557838558821251A722307B0C7559608549
:2054000057838558821251A7228583578582587559003078098557838558821251A722857B
:2054200083578582587559203079098557838558821251A722858357858258755940307A33
:20544000098557838558821251A722858357858258755960307B098557838558821251A7F1
:2054600022124DC39063B0E0F55775686075A060755800A85808E55713D8FD5035E558C4E8
:205480002304F8E2FE54C07029758363E558232324E0F582795AE0F7A309B95DF975F0003D
:2054A000EEA2E592F7A27B92F6E5F04558F5591249C80558E558B404BA2275836075F0205B
:2054C000A42EF582E0FEA3E0F5F0EE2230040122752F007460F568F5A0E5303007092006F1
:2054E00006300503D27DC4540F75F003A49054F17302551202554C0255860255C00255FA53
:2055000002563402566E02569D0257110257850257E3207D087554007555008006755440F9
:2055200075550220080A8554599051FB1251A72285555912513612516378809058CB12588C
:20554000D95008A8549051FB1258A322207D08755400755510800675544075551220090A2D
:2055600085545990520B1251A72285555912513612516378A09058CD1258D95008A854905A
:20558000520B1258A322207D087554007555208006755440755522200A0A85545990521B49
:2055A0001251A72285555912513612516378C09058CF1258D95008A85490521B1258A3227B
:2055C000207D087554007555308006755440755532200B0A85545990522B1251A72285555E
:2055E0005912513612516378E09058D11258D95008A85490522B1258A322207D08755400A1
:20560000755500800675544075550220080A85545990523B1251A722855559125136125189
:205620006378809058D31258D95008A85490523B1258A322207D087554007555208006751E
:205640005440755522200A0A85545990524B1251A72285555912513612516378C09058D584
:205660001258D95008A85490524B1258A32275540075550020080A85545990525B1251A7F9
:205680002285555912513612516378809058D71258D95008A85490525B1258A322207D08F7
:2056A000755400755500800675544075550220080B85545990526B1251A7801B8555591260
:2056C000513612516378809058CB1258D95008A85490526B1258A3207D0875542075551178
:2056E000800675546075551320090A85545990527B1251A72285555912513612516378A086
:205700009058CD1258D95008A85490527B1258A322207D0875540075552080067554407555
:205720005522200A0B85545990528B1251A7801B85555912513612516378C09058CF12588E
:20574000D95008A85490528B1258A3207D087554207555318006755460755533200B0A85B3
:20576000545990529B1251A72285555912513612516378E09058D11258D95008A8549052B7
:205780009B1258A32275540075550020080B8554599052AB1251A7801B8555591251361237
:2057A000516378809058D31258D95008A8549052AB1258A3755420755521200A0A85545917
:2057C0009052BB1251A72285555912513612516378C09058D51258D95008A8549052BB1233
:2057E00058A32275540075550020080B8554599052CB1251A7801B855559125136125163B0
:2058000078809058CB1258D95008A8549052CB1258A375542075551120090B855459905280
:20582000DB1251A7801B85555912513612516378A09058CD1258D95008A8549052DB1258CB
:20584000A3755440755522200A0B8554599052EB1251A7801B85555912513612516378C00D
:205860009058CF1258D95008A8549052EB1258A3755460755533200B0A8554599052FB1284
:2058800051A72285555912513612516378E09058D11258D95008A8549052FB1258A322E2C6
:2058A000540F22740128F9E3543FF3790C740428F8740493F2A308D9F822E493F55EA3E45B
:2058C00093F55F126A1BE55EA2E7227EDFBEDFDF5FEF5FF7BFFBBFFDFF12589FFF1258BA3E
:2058E0002230040122C205C278E530300709200606300503D278C4540F75F003A49059010E
:205900007302592202593C02595602597002598A0259BB0259EC025A2B025A5C025A8D0218
:205920005ACB2078057559808003755982125136125163755800125B16025B07207805755F
:2059400059908003755992125136125163755811125B16025B072078057559A080037559FB
:20596000A2125136125163755822125B16025B072078057559B080037559B2125136125136
:2059800063755833125B16025B072078057559808003755982125136125163755804125B62
:2059A000162078057559908003755992125136125163755814125B16025B07207805755961
:2059C000A080037559A2125136125163755825125B162078057559B080037559B2125136A9
:2059E000125163755835125B16025B07755980125136125163755806125B16755990125134
:205A000036125163755816125B167559A0125136125163755826125B167559B012513612B8
:205A20005163755836125B16025B07207805755980800375598212513612516375580712C5
:205A40005B162078057559918003755993125136125163755817125B16025B0720780575B9
:205A600059A080037559A2125136125163755828125B162078057559B180037559B31251E0
:205A800036125163755838125B16025B07755980125136125163755809125B1675599012A8
:205AA0005136125163755819125B167559A1125136125163755829125B167559B1125136D1
:205AC000125163755839125B16803C75598012513612516375580A125B16755991125136BC
:205AE00012516375581A125B167559A212513612516375582A125B167559B31251361251B0
:205B00006375583A125B1630070B200608200505D2050258E922E5592354602480F8E558D4
:205B2000F222C02FC27B125461125BC3124D16D27B125461D02F125B47E52054C3B4C2035D
:205B40001266C175A8FB2230790122301174AA30E520F5F053F003C4540C45F0700A7800FC
:205B600090F601531A0F8047B40D0A780B90F617531A0F803AB40E0A781690F62D531A0FB1
:205B8000802DB40818782190F6438AF053F00FEAC4540FC395F05017EAC4FA8012B4090798
:205BA000783390F6678008B40AB4785790F6AFE493B51A028007A3A308B880F322AB181210
:205BC0005F9622C204126667B90F2AE5255403704CE530540FB5500A200707123C76123B34
:205BE0004F22D22A53200C5325FC855030C231C205125C6822E530540FB5500280CD125C54
:205C00009520E70280DCD207C20653300FE550C44230D231753920D205125C6822E53054E3
:205C20000FB550134320C05320FCE525540342205325FCC23180E0F9125C9520E703025BBE
:205C4000E24320A05320ACE525540342205325FC53300FE550C4423080B890517F7409F007
:205C60002290517F7408F022124A70125C5A1254CC123C0C123C76123B4F12652730070EB1
:205C8000E52054CBB48202800512650F80031264DC125C6122905CADE5502393F55EE550CB
:205CA000230493F55F891F126A1BE55E227480B480D900E9003480C90000003480C900004E
:205CC000000000E530905CF093F5F030F006758240125CFB30F106758250125CFB30F20696
:205CE000758260125CFB30F306758270125CFB2201020408030C0F030C0F0F7461F568F548
:205D0000A0F58378F0790AE2F0080582D9F92275686075A060E561C4232401F87901E2547F
:205D2000FEF5F07A04E3A2E0E5F092E0F3E92420F9DAF27B0E755012E561C4232550F8E295
:205D4000F5F0A9507A04E5F0F3E92420F9DAF70550DBE5123DA22275686075A060E56E54A7
:205D60007F905E5393700122905D71E56E547F2373220022002200220080288038220022F7
:205D800000220022002200803E803C803A8050804E804C804A8048804680448042804080E1
:205DA0003E803C755001755104125DFC0551125DFC123DA222755001755106125DFC0551C7
:205DC000125DFC123DA222755001905DDCE56EC3940B93F551125DFC123DA2220203019014
:205DE0005DF1E56EC3940E93F550125E3B123DA22212131714181519161D1E1FE561C423D4
:205E00002550F8E2F5F07A04A95090FA8CE5519355F0601490FA8CE55193F5F0E345F0F370
:205E2000E92420F9DAF6801290FA94E55193F5F0E355F0F3E92420F9DAF622E561C4232589
:205E400050F8E2F5F07A04A950E5F0F3E92420F9DAF72200000000010100000000000101D7
:205E6000010101010101010101010101202F0B7888E6B5580908E6B55904125EE922125ED5
:205E8000E9C2AC75D00875686675A06674E02531B50A028004F50AF30985585C85595D75CD
:205EA0005E01755F00126824855C5E855D5F855F5A1268D91268D9E55A5403C423F55BB42C
:205EC0002008E55F6010E55B800CB46009E55FB47F028002E55BF309E55FF30975D01830F9
:205EE0002E04C22ED299D2AC227888E558F608E559F622C2AC75686675A06675D00874B047
:205F00002531B50A028004F50AF3097401F309302604747F8001E4F30975D018302E04C24B
:205F20002ED299D2AC2275686675A066750A00AAD0C2AC75D00820921A74B02531F3097400
:205F40007BF309E4F30920130A2033077440F309E4F30920120A3026077401F309E4F309D9
:205F6000201411E545600D74E02531F3097440F309E4F3098AD0302E04C22ED299D2ACE595
:205F800008B50901221278D3E508B50902800075080075090022C2AC75D00875686675A05E
:205FA0006674C02531F50AF309E51BF30975D018302E04C22ED299D2AC22C2AC756866751A
:205FC000A06675D00874B02531B50A028004F50AF3097440F309303304747F8001E4F30949
:205FE00075D018302E04C22ED299D2AC22C270C23275686375A063E52054C3B4C202D27033
:206000007900E9C42401F8E230E51120E40E20E60B540FF2E9C42405F87405F209207005E6
:20602000B908DF8003B904DAC232789CE4F608B8A6FB22C2AC75686675A06675D00874FE56
:20604000F30975D018302E04C22ED299D2AC22C2AC75686675A06675D00874B02531B50AD8
:20606000028004F50AF309E552B50C02800AF50C7464F309E552F309E50B600A750B0074C5
:2060800065F309E4F3097406F309E553F3097426F309E554F30975D018302E04C22ED29930
:2060A000D2AC22C27075686375A0637900E9C42401F8E230E50B540FF2E9C42405F8740575
:2060C000F209B908E8C232789CE4F608B8A6FB22C23275686375A06378017905E2547070FE
:2060E000037405F3E82410F8E92410F9B881ED22C2AC75686675A06675D008750A0074F063
:20610000F3097441F309E531540FF3097410F309E550F309751851055F055F055F755D00D0
:2061200075D018E6C0E0255DF55DD0E00875D008F309D55FEBE55DF404547FF30974F7F321
:206140000975D018302E04C22ED299D2AC22755012755100755208755F011260F022201681
:20616000012275F005E553A4F5F090619A7854E5F093A3F608B859F775686475A064A854B3
:20618000E2A955B900028004031980F755568557F0842558F55412614E220900FF02000A95
:2061A00000FF02000B00FF02000C00FF0200130101010006020101000500FF020006060390
:2061C0000100060403010007001F010008000F010011007F010012007F0100130001010039
:2061E00010007F0100130301010013020101000D007F01000E00FF02000F00FF01400400F1
:20620000FF020000007F010001007F010002007F010003007F010020160122124DC3906309
:20622000B0E0F5F0E552232390622C7320F00D2220F1092220F2052220F30122E553700346
:2062400002630F53520375F006E55314A4F5F09063477854E5F093A3F608B85AF77568608D
:2062600075A060E552C423F55DE5546003026291E555255DF8E2A956B90002800403198038
:20628000F7555725588559F084F554755F01026327E554B40209755D00755E000262B875B4
:2062A000836374B12552F582E023F5F090633993F55DE5F00493F55E755F0075686075A007
:2062C00060E552C423F5502555F8E2A956B900028004031980F75403F55AE5572550F8E2A5
:2062E000F55B08E2F55C1268A5E55C540FF554E55CC4540FF555E55B540FF556E55BC4540F
:206300000FF557E55A5403F558755F05026327906100E552C42582F5827854E0547FF6A3B8
:2063200008B85DF7755F09755012755100906421E55393F5531260F022010001800200029D
:20634000800100020001000002007F0001001000FF4001001100FF4001000104030001008D
:206360000106030001010E06040001010E00080001020E02060001010F040C0001020F068F
:206380000A0001000102010001000103010001000101010001001200FFFF02001300FFFFC0
:2063A00002001700FFFF02001400FFFF02001800FFFF02001500FFFF02001900FFFF02006A
:2063C0001600FFFF02001D00FFFF02001E00FFFF02001F00FFFF02001A007F0001001B0098
:2063E0007F0001001C007F000100FFFFFFFFFFFFFFFF010203040506FFFFFFFF07FFFFFF74
:20640000FF08FFFFFFFF09FFFFFFFF0AFFFFFFFF0B0C0D0E0F101112131415161718191A46
:206420001B00090A0B0C0D0E13181D222728292A2B2C2D2E2F3031323334353637C2AC7590
:20644000686675A06674902531FB75D018789279007A18E6601F135015F5F075D008E51B1D
:20646000F309E51AF309E4F30975D018E5F0090AB908E38004EA2408FA790008B89CD475AA
:20648000D00874B02531F50AF309747BF309E4F30975D018302E04C22ED299D2AC7892E45E
:2064A000F608B89CFA22E4F502F505F50DF4F506F5072275839079011264C9E4F07583C0BD
:2064C00079FE1264C9E4F4F022E9F023F978191278EDD8FBB9010122B9FEEE2275686375F3
:2064E000A063E478007900F2E82410F809E9B408F622787079C07583A0C22BE82490F0E0E6
:20650000C6F446F4F76002D22B0809B877ED2275686375A063E478007900F2E82410F80946
:20652000E95403B908F42275686375A0637800E4F208B880FB22C2ACE47800F608B806FB60
:20654000C222202605202502C223C237C232F54DF549F54A75020075030075040075050052
:20656000789CF608B8A6FB7583637800E8C404F582E054F0B4A019E4F0E8C42405F582E421
:20658000F07D007E00E804C454F02403FF1249B708B808D8758600758700C25922D22F759A
:2065A000A8F190517F7409F015821582E00582E0124A70E47892F608B89CFB1278D3126525
:2065C00036C2AC850100C230C25B53300FC231532018123C0C5324A3532703E47828F608FF
:2065E000B82EFB7835F608B843FB7543FF1265271264DC2275D018E530540FC3940B4004D5
:20660000D2048002C2041254CC123C0C123C76123B4F1265273007115320FCE52054CBB443
:206620008202800512650F80031264DC90517F7408F078007920E4F608D9FC7870E4F4F6AC
:2066400008B878FBC298C2998501008509087506FF7507FF750BFF750CFF75A8FB124D16B5
:2066600075280075290022E530540F90668B93F5F0C4540F2470F8E5F0540FF9E613D9FD99
:206680005003790F22E530540FF9220102030414152122232425C2D578C079707A00E66010
:2066A0001A13501330D50E90FA94EA93F5F056F6E5F0F447F7D2D50ABA05E60908B8C7DCA2
:2066C0002275686875A0687800E4F2D8FD05688568A0E568B46CF290640DE0C33375F0D846
:2066E000A4E5F0240175F004A485F014F51575120075130075686375A063784579047405E2
:20670000F2E82410F8D9F779047841E2548FF2E82410F8D9F62212678275686375A0637886
:2067200000E8C42401F9E3548FF3E8C42405F97405F308B808EB2275A064780090674DE4AE
:2067400093F208A3B814F8D251532301221717171700C800010A8096001E40800014285AD0
:206760000075A0649067757880E493F208A3B88DF875221C2200001C0704010000001C00D2
:20678000001C123B1A90FF02C3123AE0123B27C3123AE01278ED753850D22D229064007892
:2067A0008D75F000E025F0F5F0A3D8F8227D7FE55623FEE55754F02413FF1249B722E47DD5
:2067C00040FEFF1249B77D1F7EFF7F011249B77DC0FE7F021249B77D7F7EFF7F131249B7D4
:2067E000FD7E047F041249B77D7F7EFF7F051249B77D7F7EFF7F061249B790E0007401F091
:20680000227D817E00E55754F02413FF1249B7124998E55754F02417FF7A001250FDEE603E
:2068200002DAF822C3E55D255FF55DE55C355EF55C22C3E55D955FF55DE55C955EF55C224E
:20684000C3E55D255FD4F55DE55C355ED4F55C22C3E55DB55F07E55CB55E02D322C32275A9
:20686000F000E55E700575F008800C54F0701A75F004E55EC48012E55F700475F010225404
:20688000F0700675F00CE55FC420E7052305F080F822E55C255FF55CE55B355EF55BE55AE3
:2068A000355DF55A22C3E55C955FF55CE55B955EF55BE55A955DF55A22C3E55AB55D0CE562
:2068C0005BB55E07E55CB55F02D322C322C3E55F33F55FE55E33F55E22C3E55E13F55EE548
:2068E0005F13F55F22F55AC394644003749922E55A75F00A8485F05AC454F0455A22E55B2A
:2069000004F55B700BE55A04F55A6008540F6008C3C27822D3D27822D27822E55B14F55B75
:20692000B4FF16E55A14F55AB4FF028008540FB40F07D27822D3D27822C3C27822C278E599
:206940005C04F55C700EE55B04F55B7008D278E55A04F55A22540F70FBD27822C278E55C49
:2069600014F55CB4FF19E55B14F55BB4FF028008540FB40F0AD27822D278E55A14F55A225B
:206980007910E55D33F55DE55C33F55CE55B33F55BE55A33F55AE55BC3955FF55BE55A9543
:2069A0005EF55A500DE55B255FF55BE55A355EF55AD3B3D9CDE55D33F55DE55C33F55C22BE
:2069C000855FF0E55EA4F55C85F05B855FF0E55DA4255BF55BE5F0500104F55A22E55EC4AF
:2069E00054F0F55EE55FC4540F455EF55EE55FC454F0F55F22E55FC4540FF55FE55EC454C3
:206A0000F0455FF55FE55EC4540FF55E22855F5E755F0022855E5F755E0022EF30E40775C1
:206A20005E00755F002230E307C2E3FF126A0DEF30E207C2E2FF1269DDEF30E10AC2E1FF0C
:206A40001268CD1268CDEF30E006C2E0FF1268CD22EF30E407755E00755F002230E307C2EA
:206A6000E3FF126A14EF30E207C2E2FF1269F5EF30E10AC2E1FF1268D91268D9EF30E00632
:206A8000C2E0FF1268D922EF75F06484FEE5F01268E5FF2275F000E55A700575F008800C3F
:206AA00054F0702D75F004E55AC48025E55B701775F010E55C700475F0182254F070127519
:206AC000F014E55CC4800A54F0700675F00CE55BC420E7052305F080F822C3E55C33F55CAE
:206AE000E55B33F55BE55A33F55A22C3E55A13F55AE55B13F55BE55C13F55C22E55AC454CB
:206B0000F0F55AE55BC4540F455AF55AE55BC454F0F55BE55CC4540F455BF55BE55CC45498
:206B2000F0F55C22E55CC4540FF55CE55BC454F0455CF55CE55BC4540FF55BE55AC454F001
:206B4000455BF55BE55AC4540FF55A22855B5A855C5B755C0022855B5C855A5B755A00229E
:206B6000EF30E409C2E4FF126B4C126B4CEF30E307C2E3FF126B4CEF30E207C2E2FF126A35
:206B8000FCEF30E10AC2E1FF126ADA126ADAEF30E006C2E0FF126ADA22EF30E409C2E4FFD2
:206BA000126B56126B56EF30E307C2E3FF126B56EF30E207C2E2FF126B24EF30E10AC2E1B6
:206BC000FF126AEB126AEBEF30E006C2E0FF126AEB22E55CF4F55CE55BF4F55BE55AF4F587
:206BE0005A22752F00E55F30E705D278F4F55FC333C4540FF55E740F955EB40F04D2797417
:206C00000EF55EE55F30E20D307905755A018010755A03800B307905755A008003755A0274
:206C2000C4232354C0F55B755C00AF5E126B99307803126BD222752F00E55A30E20B44F89A
:206C4000F55A126BD2D27880045407F55A126A94E5F0C394164005D27975F0157415C395E1
:206C6000F0C4035478F55F741430790104C395F0FF126B99E55C5407455F307801F4F55F79
:206C800022785AE47906F6D9FD85655578667956126CB4126CB4795F126CA1F719B959F870
:206CA000227856E4C555C44675F00A84F6E5F008B85AF322E6C4540FF709E6540FF7090891
:206CC00022755C00755D008DF0EFA485F05EF55F8CF0EFA4255EF55EE5F0355DF55D8DF09D
:206CE000EEA4255EF55EE5F0355DF55DE4355CF55C8CF0EEA4255DF55DE5F0355CF55C22F2
:206D0000C0A875A8EB75D018124A70906E58123D00123B4F75320F90E0087410F075820000
:206D2000E020E1FC90F000F0906E527568E475A0E47A0378047B00E4F208F218DBFAE49354
:206D4000A3F550E493A3F551E551F208E550F218DBF6DAE1753C0A307011126D91207D09CE
:206D6000126DB3123B4F126DD380EF7538108004E5387011053253320F753810126DB312D9
:206D80003B4F126DD31264F2302BE5124A70D0A822C27DE53C123AD5940450028012753C5B
:206DA00000207F06053253320F22153253320F22D27D2278BDAF32126A87EFC4540F600440
:206DC000243080027420F608EF540F2430F6087420F622E47D40FEFF126E46AD007E227FCB
:206DE00001126E467D007E007F02126E467D7F906E68E53293FE7F13126E3A906E78E532A7
:206E000093FE7F23126E3A7E047F04126E467D007E887F05126E46906E88E53293FD7E86BC
:206E20007F06126E3A906E98E53293FD7F16126E3A90E00074FFF0A3F0227C081249B7EF7A
:206E40002420FFDCF7227C101249B7EF2410FFDCF7228000400001002054455354494E4746
:206E6000204249542D20202002020408102001020408102040808000000204081020010286
:206E800004081020408080000505050505050303030303030303010005050505050503031B
:206EA0000303030303030100752F0053210F1270588036752F0153210F1270588027752FBB
:206EC0002153210FF554126F6C801E752F0180F1752F6053210FF554126EFA8008752F406E
:206EE00080F112726D53210F22540FC313906EF593906ECB7300DD171A1A12794550012225
:206F0000207F0512748880031274D8E551703C307F0FE550540F8530F053F00FB5F0298061
:206F20000EE550540FF530123C0C12723ED27FD22A12724B500122907ABE1273C3127971CF
:206F400050B8127A0250F62275510912792E4014127ADE12792E400C1264F2302BF5127AA4
:206F60000250F0221279454002808F22C27C1279455003740822907A4C1273C3C27E127407
:206F800088E5516029207C04D27C80E212792E4016127ADE12792E400E1264F2302BF51210
:206FA0007A0250F074082212794550C080F690618AE0F5507568808568A078007480F20831
:206FC0007420F2089061801273E1E550C4540F04FF7420F208E52113F55AE433F2DF089077
:206FE0006190F0A3740DF008E55AB808EA7420F21278ED78C77466F6087401F6E550C454DF
:207000000F244308F643A882D23053210F12723EC050C030E550540FF530123C0C12797135
:20702000400F53A8FDC230D030D050123C0C026F6C127A025002801108E630E0E0D030D0A1
:207040005053A8FDC230740422D030D050123C0C53A8FDC230740822E530540F907A109335
:207060004521F521C47AFF130A50FCEAC4F5501278B8240EF582E01278AC7568618568A02F
:2070800079F07F0AE0A3F309DFFA907A847800C3123AE0123AFB1278ED7B877CF053A8DDAD
:2070A000C23078007487F2089061F0E0A3F208123AFB1278ED780074C0F208D3123AE0129E
:2070C00078EDE42C758361F582E0F55E758290F0A3740DF078C9EBF678C77466F6087401FF
:2070E000F6755D04D230753C0043A8A21278D3E53C20E709B41000401854F08007B4F1006A
:20710000500F440F12716FF55E7583618C82F0808C1264F2302BD5127A025002803908E6F6
:20712000541E603B20E21420E32220E427740453A8DDC2303078030272D2220CBCF9027C48
:20714000F8907A1FEC540F93FB02709D1CBCEFF17CF080ED125CC353A8DDC2307408227880
:20716000C6E630E08774207583618C82F080CCC4C55E24E09071DE93255E30E704245180A5
:2071800007B45100400224AF90718D9322204142434445464748494A4B4C4D4E4F50515240
:2071A000535455565758595A6162636465666768696A6B6C6D6E6F707172737475767778EF
:2071C000797A303132333435363738392623213F2E2C3A3B27222A2B2D2F3C3D3E5F0041E6
:2071E000484000003F470000494A444B434C35363738393A3B3C3D3E45464D4E4F420001D9
:2072000002030405060708090A0B0C0D0E0F101112131415161718191A0000000050001BA5
:207220001C1D1E1F202122232425262728292A2B2C2D2E2F30313233340000000000E55031
:20724000540F907A10934521F52122E550C4540F907A2893FFF4C445215FF52154F0600227
:20726000C322907A741273C31278F6D3222078030272D2127945500122907A6C7800C31207
:207280003AE09061801273E17420F21274D8E5517025D22AE550540FF530123C0C12724B6C
:2072A0004014907ABE1273C31279714004D27F80C2127A0250F22212792E40B7127ADE1279
:2072C000792E40AF1264F2302BF5127A0250F074082212794550012212793A5009907A8DFC
:2072E0001273C302737A307802803E907A4C1273C3C27E127488E5517029907A9D7800C352
:20730000123AE09061801273E1907AA4C3123AE0127971400280BB127A0250012208E65411
:207320000260ED1279455001221278AC7568618568A079F07F0AE309F0A3DFFA907AA6C3FD
:207340007800123AE09061F01273E17420F212772CE55160028007127687E551602D12798B
:207360002E4007207C04D27C80E4755107C27C12792E50030272D2127ADE12792E40F5127F
:2073800064F2302BF5127A0250F022E550C4540F907A28935521F52154F0601D907ABE120F
:2073A00073C312797140028007127A0250F44012E5502410F5500272D2907AAE1273C312A8
:2073C00078F6227480F568F5A07800F208C3123AE01278ED780074C0F208123AE01278ED16
:2073E000227568808568A0E0A3B40D0122F208B809F51278ED780074C080F27800F2081251
:207400003AFB1278ED2212784B40211279AF401CB4021A1279EA40141278E312785F400C97
:207420007D041279C440057D0A9061802275510622C083C0827D0F1279C440477F0A9077B8
:20744000D3E493A3F57D1279AF4038B57D32DFF17D1C1279C4402C1279EA4027307E129067
:207460007A6CC37800123AE09061801273E17420F21278D312785F400A7D031279C4800380
:20748000755105D082D08322127406403B1279AF4036F0F552E0B55227A3DDF1B40D2612F4
:2074A000743140241279AF401FF556E55430E702E556F0307E05F55002751875510080088D
:2074C0007551088003755105027678D0E0755109800375510502767812740640F8E0A3F5A7
:2074E000521279AF40EFB552E4DDF2B40DE412743140E21279AF40DDF556E55420E703852F
:207500005456E556307F11C0E0540FF552E550540FB552B7D0E0F550B550B21278B8E55003
:20752000F0F552E0B55245A37D1FE5543392D520D5027D031279AF409CF0F552E0B5522CFF
:20754000A3DDF130D5030275F11279AF4087547FF556E554540103F55B4556F0F552E0B5E3
:20756000520AA31279AF400FF0F552E0B55257A37D027C021279AF402DF0F552E0B5524663
:20758000A3DCF11279AF401E547F455BF0F552E0B55233A31279AF400DF0F552E0B55226B1
:2075A000A3DDCF1279AF4054543CF556C083C082E554540FC31390768593C5564556D082B6
:2075C000D083F0F552E0B55222A31279AF402D54CFC5565403C44556F0F552E0B5520CA30D
:2075E0007D101279AF4015F0F552E0B5521CA3DDF1307D197D809064001279AF4027F0F587
:2076000052E0B55205A3DDF180080276757D801279C41278C590E008F0FC90FFFFF07E0843
:207620007D001279AF4051F5521279AF404AF55390E404F0A3E552F01279AF403BFF90E455
:2076400004E553C4F0A3EFF0DDD8DED6EC04DBC51279EA40231278ACE582F8756861856827
:20766000A07980E309F2F552E2B5520908B40DF375510080037551087568408568A0127952
:207680008E12790C22418212740650060277290277261278ACE0A3F5521279AF40EEB5524E
:2076A000EEDDF2B40DE912743140E11278B87D20E0A3F5521279AF40D3B552D3DDF27D80EF
:2076C000906400E0A3F5521279AF40C0B552C0DDF21278C590E008F0FC90F000E07E087D06
:2076E0000090E404E054F0F553A3E0F5521279AF4037B5523190E404E0C4540F4553F55295
:207700001279AF4024B5521EA3E0F5521279AF4018B55212DDCBDEC9EC04DBB81279EA40AA
:2077200008755100800375510702767812780B7F021279A51279D61278279077BF1277FE96
:207740001278ACE0A3FF1279A5BF0DF79077C41277FE1279D612782C1277FE1278B87E20AE
:20776000E0A3FF1279A5DEF87E80906400E0A3FF1279A5DEF81278C590E008F0FC90F000D4
:20778000E07E087D0090E404E054F0F552A3E0FF1279A590E404E0C4540F4552FF1279A52C
:2077A000A3E0FF1279A5DDDDDEDBEC04DBCA1279D6755100127994400375510602767800CA
:2077C000400001FF202020202020200000A0C000000000526F6C616E6420533130000000F5
:2077E00000000000000000000000000000000000000000000000000000FF05A0C0FFE493AF
:20780000A3B4FF0122FF1279A580F312790512798812799450FB1278DF1278E31279991234
:2078200078E31278E3800E12790580F01279051279991278DB12799F7F161279A51278CF91
:2078400078037430F27FA51279A5221278FE12798812799450FB1278DF1278E31278E375E4
:2078600068408568A078017414F278037410F21278FE7803E4F278017484F27F007E8F78AF
:2078800001E220E609DFFADEF8755102801C1279AF4017B4160280F6B4A50C78037420F2AA
:2078A00074A51279BFC322755103D322E55054F02440758361F58222E55054F0232480753E
:2078C0008360F58222E55054F00324107B08227E0180127E0B800E7E14800A7E1D80067EF4
:2078E0007C80027EA07F72A4DFFDDEF9227F0000000000DFFA22780A1278E3D8FB22127919
:207900000C7414F22212790C7411F2227568408568A07801A4E4F2A4E4F2A4E4F2A47440A6
:20792000F2A4740CF2A47416F2A47416F2227568408568A07803E2A2E1227568408568A087
:207940007803E21322C27A12792E501B1264F2302B06127A02500122207AEC907A3C12731A
:20796000C3D27AC27B80E01278D312792E40E9C32212792E40081264F2302BF5D3221278FF
:20798000D312792E50EBC32278037410F22278037418F2227801E233227801740BF22278D9
:2079A000017403F2227801E230E0FC18EFF2227801E230E405755101D32230E1F418E27812
:2079C00002F2C3221279AF4002DDF9227802E2F55208E2F553221279CC7410F2AF5212790A
:2079E000A5AF531279A51278CF221279CCE4F21279AFB552081279AFB55302C322755104CC
:207A0000D3227F0378C0E6087004DFFAC322D3221020408030C0F030C0F0F030C0F0F087AB
:207A2000C0C1C2C3C4C5C6C7EFDFBF7F2020202057726F6E672051442020202020202049B3
:207A40006E736572742051442020202020202020436865636B205144202020202020496C3D
:207A60006C6567616C2051442020202080204C6F6164200D204C6F616420636F6D706C653F
:207A800074652020804E616D65203A200D2057726974652070726F746563746564804B69FC
:207AA0006C6C200D203F802053617665200D205361766520636F6D706C657465202020205E
:207AC000204368616E67652051442020202020436F70792070726F74656374656420E55110
:207AE00060151423FF907AF893FEEF0493F5828E831273C31278F6227B0A7A5C7A5C7B1A8A
:207B00007A5C7B2A7B3A7B4A7A2C2020492F4F204572726F7220312020202020492F4F20C1
:207B20004572726F7220322020202020492F4F204572726F722033202020202056657269CF
:207B40006679204572726F7220202020492F4F204572726F72203420202043D01890618C4F
:207B6000E4F55DF0202171302A6EE530540FB40700500D906001E0C2E0F0A3743CF0805857
:207B8000B40A2E906001E0C2E0F0A37429F0906021E0C2E0F0A37435F0906041E0C2E0F004
:207BA000A37441F0906061E0C2E0F0A3744DF08027906001E0C2E0F0A37430F0906021E034
:207BC000C2E0F0A37448F0800F402EC290540E03907BF193907BD8731287D780EC7538148E
:207BE000127ED080E41281F180DFD27C1284CD80D800050D031203030353A881C23090E0C7
:207C000000E4F0A3F0758206F0D290D295D297755D00E530540FF55F908B4E93F55C906102
:207C20008CE0540FF55E302103027CDA30E012432F0CE55C128DFC307F07906001E0543FE0
:207C4000F0E55FB407005003027CDAB40903755C02055C055DE55E30E11C207F0B432F0C9C
:207C6000E55C128DFC307F0E906001E0543FF0906021E0543FF0E55FB40A5F055C055DE59A
:207C80005E30E223207F0B432F0CE55C128DFC307F15906001E0543FF0906021E0543FF0C1
:207CA000906041E0543FF0055C055DE55E30E32A207F0B432F0CE55C128DFC307F1C90602E
:207CC00001E0543FF0906021E0543FF0906041E0543FF0906061E0543FF0C27F128D097526
:207CE000A08090FF9274407B08123B0690CFFAE55F93F55AE55FB407004003027D8CE55EAA
:207D00007003027EC6E55AC4F5501278B88582507F00AE827D607B2012AD9FE550C3137FBA
:207D200000FE7D617B1012AD9FE55FB404005003027EC6E55A04C4F5501278B88582507F85
:207D400000AE827D607B2012AD9FE550C3137F00FE7D617B1012AD9FE55FB4062C7F007EA7
:207D6000C07D607B2012AD9F7F007E607D617B1012AD9F7F007EE07D607B2012AD9F7F0017
:207D80007E707D617B1012AD9F027EC6B40900505BE55E54056024E55AC4F5501278B88551
:207DA00082507F00AE827D607B2012AD9FE550C3137F00FE7D617B1012AD9FE55E540A700C
:207DC00003027EC6E55A04C4F5501278B88582507F20AE827D607B2012AD9FE550C3137F46
:207DE00010FE7D617B1012AD9F027EC6B40969E55E5401602C7F007E807D607B2012AD9FCB
:207E00007F007E407D617B1012AD9F7F007EA07D607B2012AD9F7F007E507D617B1012AD76
:207E20009FE55E54027003027EC67F207EC07D607B2012AD9F7F107E607D617B1012AD9F6A
:207E40007F207EE07D607B2012AD9F7F107E707D617B1012AD9F806EE55E606A30E0167F6B
:207E6000007E807D607B2012AD9F7F007E407D617B1012AD9FE55E30E1167F207EA07D6026
:207E80007B2012AD9F7F107E507D617B1012AD9FE55E30E2167F407EC07D607B2012AD9F87
:207EA0007F207E607D617B1012AD9FE55E30E3167F607EE07D607B2012AD9F7F307E707DE5
:207EC000617B1012AD9F128D6490618CE054F0221264F27876E644FE906800F053A881C2EE
:207EE000309089B51273C3E55DC4F5501278B8C2E72402F582E0FA858353858252C2308564
:207F00005383855282EAF0209206207C03027FCBC05D123D4712AE9ED05D209206207C0320
:207F2000027FCB743029906192F0A3740DF078C97444F6D230209206207C03027FCB753C5C
:207F40000043A8A21278D7209206207C03027FCBE53C20E70FB410004019EA04B4680050E2
:207F6000DDFA8099B4F100500AEA14B4180040CEFA808A209205207C028050E538906800FC
:207F8000701D7538147876E644FEF4600CF4F550E0B5500875380C801F7550FFE550F012A4
:207FA00064F2309202C27C302B9A127A02401F78C6E630E005753814801A209205207C029E
:207FC0008009128980C37006027F447408C353A881C230221264F27876E644FC906800F0CC
:207FE00053A881C2309089E31273C378C97442F6E55DC4F5501278B8C2E704F582E01392AC
:208000007F85835F85825EC230855F83855E82E0A27F92E0F020214B302A4890618CE0FE6B
:2080200020E009906001E0A27F92E0F0E530540FFFB40700402DEE20E109906021E0A27F3A
:2080400092E0F0EFB40A00401AEE20E20A906041E0A27F92E0F0EE20E309906061E0A27FDD
:2080600092E0F09089F37F40D295C297307F099089F67F20D297C29512AE9E74C07E0012CB
:20808000896AD230209206207C0302811D753C0043A8A2209206207C0302811D1278D7E579
:2080A0003C20E70AB410004012307FE18008B4F1005008207FD7B27F028007209205207CC5
:2080C00002805AE53890680070207538147876E644FCF4600FF4F550E0B5500B75380C30D5
:2080E000E02580257550FFE550F01264F2309202C27C302B9E127A02402678C6E6540360BB
:208100000B75381430E002801D027ED0209205207C028009128980C370060280937408C30E
:2081200053A881C230221264F27876E644FD906800F053A881C2309089C51273C378C97401
:2081400042F6906483E033927FC230906483E0A27F92E7F09089D5207F039089DC12AE9E96
:20816000D230753C0043A8A2209206207C030281E81278D7E53C20E70AB410004011307FA6
:20818000E18008B4F1005007207FD7B27F80BA209205207C028051E538906800701D753824
:2081A000147876E644FDF4600CF4F550E0B5500875380C801F7550FFE550F01264F23092A5
:2081C00002C27C302BA2127A02402078C6E630E106753814027FD4209205207C0280091233
:2081E0008980C370060281687408C353A881C2302253A881C2309080007480F0A37420F0FA
:20820000E582B408F71278ED209206207C0302841C7568808568A0908A9974507B01123BAA
:2082200006906483E0F55A33927F75520175510053A8817568638568A078B09084A5E4931F
:20824000A3F208B40EF89084B9E493A3F208B40EF8906483E55AF0307F030282DAE55A90A7
:208260008AA19304B4080040022403F55B7568638568A074B0255BF87401F274C4255BF847
:20828000E4F2908423E55A9375F008A4F55C9089F9E55BB40D004003908A21E55C85825F65
:2082A000255FF582E5833400F58374407B017568808568A0123B06908A49E55BB40D00409E
:2082C00003908A71E55C85825F255FF582E5833400F58374487B01123B06209206207C0378
:2082E00002841C207F06753C0043A8A07F8075530090E0007E00E020E007DEFA755300803F
:208300003B758205E030E701F4B553004002F553209206207C0302841CDFD6207F1EE55305
:20832000B55A005007D5591474208005742A7559107583637582C2F07582D6F02092062067
:208340007C0302841CE553908AA193B552028011500DE5512440F551E5529400700104F56A
:2083600052FA7583637582B07568808568A07800532F9F209206207C0302841C307E06255A
:2083800082F582C27EE0A3B40D02801EB40E051278ED8029F208BA000A207DE07414432FA4
:2083A0006080D920E7D6DAD480EF1278ED209206207C0302841C7800BA00C180DC20920594
:2083C000207C0280571278ED207F26E53C20E709B40700401C055A8007B4FA005013155A3E
:2083E000E55A30E707B4FF0304800114F55A028230209205207C0280231264F2309202C2E8
:208400007C302B15127A024016209205207C02800B128980540BC370060282EC7408C353F7
:20842000A881220002040102030400010203040001020303040000010203030400000102BA
:208440000203030400000101020203030400000101020203030404000001010102020303DF
:208460000404000000010101020203030404000000010101020202030304040000000101C6
:208480000102020203030304040000000000000101010101010202020202020303030303A3
:2084A0000304040404813D3D3D3D3D3D3D800DC03D3D0202020220200E812020202020201F
:2084C00020800DC020202020202020200EC23053A881906483E0F55820E71790E000E03071
:2084E000E0F990E005E030E701F4B5580040030285859089A21273C3E55DC4F5501278B856
:20850000C2E72402F582E0FAC05D123D47D05D743029FD75A080780074C3F208C3123AE064
:20852000123AFB1278ED780074C5F208EDF208123AFB1278ED906483E0F55830E71F1264DD
:20854000F2309202C27C302B0678C3E620E336209205207C02802E540760E3C32290E00076
:20856000E030E0F990E005E030E701F4B5580050141264F2302BE6127A0240081289805452
:208580000760DAC32290E006E4F0906900E0FFFE74C412896A90E0067403F090E001741086
:2085A000F09080007480F0A37420F0E582B408F71278ED7568808568A0908A9974507B0142
:2085C000123B06906483E0F55A33927F75520175510053A8817568638568A078B09084A5A6
:2085E000E493A3F208B40EF89084B9E493A3F208B40EF8906483E55AF0307F0302867CE5D1
:208600005A908AA19304B4080040022403F55B7568638568A074B0255BF87401F274C4250C
:208620005BF8E4F2908423E55A9375F008A4F55C9089F9E55BB40D004003908A21E55C854F
:20864000825F255FF582E5833400F58374407B017568808568A0123B06908A49E55BB40D59
:20866000004003908A71E55C85825F255FF582E5833400F58374487B01123B067F80755324
:208680000090E0007E00E020E007DEFA7553008032758205E030E701F4B553004002F55339
:2086A000DFDF207F1EE553B55A005007D5591474208005742A7559107583637582C2F07551
:2086C00082D6F0E553908AA193B552028011500DE5512440F551E5529400700104F552FA74
:2086E0007583637582B07568808568A07800532F9F307E062582F582C27EE0A3B40D02801D
:208700001EB40E051278ED8023F208BA000A207DE07414432F6080D920E7D6DAD480EF1260
:2087200078ED7800BA00CA80E502867C90E8C1E090E002E070F3A3E070EF7F33DFFEE55DEE
:2087400004FFE4D333DFFDFF908B23E530540FF55F93907A10255D934FFF90618CE04FF09B
:208760002021299064007417F0A3E582B405F7E55DC4F5501278B8C2E704F582E0540F442E
:208780004EF0EFC02FF52F128BBFD02F90618CE0F55EE55FB407004017B40A028016E55E9F
:2087A00020E005755D00802C20E105755D018024D3C22A22E55E20E005755D00801620E127
:2087C00005755D01800E20E205755D02800620E3DF755D03C3E42290E000E4F0A3F0C29029
:2087E0009089921273C3E530B407005004F555801FB40A02800E24F923F55504F5568010C2
:2088000085C0C3C6755500755601755702755803C23053A881755900908800E55993C0E091
:2088200074552559F8E612ADFDD0E012AEB51278EDE530B407000559400EB40A077404B54D
:2088400059D68004740280F77455255DF8E612ADFD12AE9E908800E55D9378C9F6D23043CC
:20886000A8A2E530540F908B2393255D2323908B327850FA93F6EA0408B853F7906900E52F
:2088800051F074C47F057E0512896A74C1AF507EFF12896A74C27FC07E0012896A7F40D214
:2088A00095C297E55DC4F5501278B8C2E7F550F582A3E030E0067F20D297C29574C07E002E
:2088C00012896A74C57F007E0412896A74C6AF527EFF12896A90E0067401F0209206207C68
:2088E00003028961753C001278D7209206207C03028961E530B407004032E53C20E720B4F6
:20890000100040287800E530B4070040077801B40A027803E8B55D0280CA055D028810B4A6
:20892000F1005008E55D60BC155D80F0209205207C02802D1264F2309202C27C302BA8122D
:208940007A02402008E6540C600520E3D780B5209205207C02800A12898054FEC370058075
:20896000867408C353A881C230227568E88568A0F8F27568E08568A07802EEF208EFF222B7
:2089800078C3E6540F2278C4E6540C2278C6E65403225245433A202020202020202020209C
:2089A00020202A20524543204B45592020202020202A80200D524543204B45592020203D33
:2089C000202020202052454320545249473D202020202020204D414E55414C0D20415554D5
:2089E0004F200D534D5020434C4B203D202020206B487A33300D31350D10100000001010E4
:208A000000080800000008080004040000000404000202000000020200010100000001011A
:208A20000018100000001018001C08000000081C000E04000000040E000702000000020768
:208A400000030100000001030010101F001F10100008081F001F08080004041F001F0404E4
:208A60000002021F001F02020001011F001F01010018101F1F1F1018001C081F1F1F081C1C
:208A8000000E041F1F1F040E0007021F1F1F02070003011F1F1F01030000001F1F1F000024
:208AA00000010101020202020303030303040404040404050505050505050606060606063D
:208AC000060607070707070707070708080808080808080808090909090909090909090998
:208AE0000A0A0A0A0A0A0A0A0A0A0A0A0B0B0B0B0B0B0B0B0B0B0B0B0B0C0C0C0C0C0C0C1B
:208B00000C0C0C0C0C0C0C0D0D0D0D0D0D0D0D0D0D0D0D0D0D0D0D0D0D0D0D0D0D0D0D0DBC
:208B20000D0D0D0001020304050600020400000204001F047F101F04FF181F087F201F0814
:208B4000FF283F04FF103F08FF207F08FF10000102030103030002010075686075A060A836
:208B600059E493F2E5822404F582E5833400F583E82404F8790CE493F2A308D9F99051EBDA
:208B8000790AE493F2A308D9F97906202A12E5822403F582E5833400F583E82403F87903F5
:208BA000E493F2A308D9F975686175A0619051DCE559C313F87910E493F208A3D9F922C2FF
:208BC0007FE530540F908BCD75F003A473028BEE028BF5028BFC028C03028C0A028C1102E7
:208BE0008C18028C1F028C2C028C39028C469051FB128C5F2290520B128C5F2290521B12B9
:208C00008C5F2290522B128C5F2290523B128C5F2290524B128C5F2290525B128CB1229055
:208C2000526B128C5F90527B128C882290528B128C5F90529B128C88229052AB128CB1903A
:208C400052BB128CC7229052CB128CB19052DB128CC79052EB128CDD9052FB128CF3228505
:208C60008357858258207F1030780C755900855783855882128B5922307A0C755940855714
:208C800083855882128B5922858357858258207F1030790C755920855783855882128B5916
:208CA00022307B0C755960855783855882128B59228583578582587559003078098557833B
:208CC000855882128B5922858357858258755920307909855783855882128B59228583578A
:208CE000858258755940307A09855783855882128B5922858357858258755960307B098559
:208D00005783855882128B59221264F2202B0122127A024001223021012290618CE030E05A
:208D200007906001E0543FF0E530540FB4070050012290618CE030E107906021E0543FF049
:208D4000E530540FB40A1C90618CE030E207906041E0543FF090618CE030E307906061E00F
:208D6000543FF0221264F2202B0122127A024001223021012290CFFAE530540F93F55A90D0
:208D8000618CE030E01BE55AC4F5501278B8A3E0543FF0E530540FB409079060A1E0543F0B
:208DA000F0E530540FB4070050012290618CE030E126E530540FB40902055A055AE55AC491
:208DC000F5501278B8A3E0543FF0E530540FB409079060E1E0543FF0E530540FB40A1C90B4
:208DE000618CE030E2079060C1E0543FF090618CE030E3079060E1E0543FF022540FC4F590
:208E000050906484E0A2E39278A2E29279307A069091A51273C3207B05C20F12ABBF127857
:208E2000C5440790E008F0A3F50A540FC4FF7E0190F000E09068007568E48568A078052030
:208E40007834E23392D5E23320D50450138002400FB2D5EEF0A3EFF0A3E583B46C02801202
:208E6000129135207F0FEE2401FEEF3400FF547F70D4028EE022E208F556E2B2E7F557187C
:208E8000E208FEE2B2E7FF18B55704EEB5560092D58F578E56E50A540FC4FF7E0290680091
:208EA000E208FAE2B2E7FB18B55704EAB556008B578A5620D50450138002400F92D5EEF007
:208EC000A3EFF0A3E583B46C028015129135207F0EEE2401FEEF3400FF547F70C3800122ED
:208EE00085820B85830C207B05C20F12ABBF9068027D687C6C7800C2D58D688568A0E2F92C
:208F0000E0A3A2D59992D58C688568A0F208E820E0E7E583B50C05E582B50B00500CB800A4
:208F2000D60D0C129135307FCE227551FF207B05C20F12ABBFE50BC39402F50BE50C94004B
:208F40002404F50C0551906C007809796CE0F50808B8000109E9B50C04E8B50B004019A337
:208F6000A3E5822409F8E5833400F9E9B50C04E8B50B0040D8028FD6129135207F571291E7
:208F80005140CD85835785825608B8000709B97003028FD689558854A3A3E0F50812915183
:208FA0004021A3A3E582B55409E583B5550418028FF7129135207F1D08B800DE09B970DA3D
:208FC000028FD6855783855682A955A85418B8FF0119028F4D22E551B405028003028F4442
:208FE000E50A540FC4440FF5517550FF74FBC0E0C051D27E0290A0E55724FCF557F58385B7
:209000005682E0FEC0E0A3E0FFC0E0E924FCF5558854F5838882E0FCA3E0FDECC39EFEED93
:209020009FFF30790CEC2EF552ED3FF553547F70078C508D5102909E7557008555838554D2
:20904000820557E557B4060280E7E0F5507F00E5502F92D5B5520280190FEFB557F17F0048
:20906000E550C39F92D5B5520280110FEFB557F08017A3E0F551A2D534008008A3E0F55102
:20908000A2D59400B553038015A3E550B552004009E0B55300400302903BA302904AC27E46
:2090A000207B05C20F12ABBFD057D056E55DC4C050F5501278B8D050C2E7F582A3E0543F83
:2090C000207E09207B04448080024440F0E5822405F582E550C39556FEE5519557FF307BDC
:2090E0000FF0A3EEF0A3E551F0A3E550F0A38004A3A3A3A3EFF0A3EEF0A3E551F0A3E550AB
:20910000F0A3E50A5430C4FF307B05E054C04FF0A3EFC4FFE0540F4FF0307A167F007E1BF4
:209120001264F2302B08127A025003D27F22DFF0DEEEC27F22C27F307B16C0D075D000AE8D
:20914000831264F2302B05127A02927F8E83D0D02289688568A0E2F5507B0008C2D5B508D6
:209160000F80270BE550C39B92D5B5080302918AEBB551EF7B00800C0BE5502B92D5B508E1
:2091800003029195EBB551F0D322A3E0F509E2A2D594008009A3E0F509E2A2D53400158232
:2091A000B509E5C3225365656B206C6F6F7020706F696E742043D01875381490610F74FFFC
:2091C000F090AAB31273C31278F675A08090B8067B017440123B06906484E0C4540F75F0A0
:2091E0000B8485F05975170053A8C1C23053210F752F00E5599091FD93909208730002051E
:20920000080B0E1114171A1D801E0293F10296890298920298C6029BE6029D4A029D580284
:209220009D69029D7A02A5141264F27876E644FE906800F0E530540FF558B40700400D9091
:20924000AAD31273C3D20D43A882802290AAC31273C378C97442F6E558F557B55802740B12
:2092600012ADFD12AE9ED230753C0043A8A2200D351278D7E558B40602802BE53C20E70CF9
:20928000B410004021E557B558DC800CB4F1005015E557B5580280CEE5579092A09380B98B
:2092A000010003020504E538906800701D7538147876E644FEF4600CF4F550E0B55008752B
:2092C0003808802B7550FFE550F01264F2302B9E127A02500712ADCF53210F2208E620E44F
:2092E0001308E6541F70EE08E630E08275381405590291E8200DAF53A8DDC230E558B55793
:2093000004D27A80064004C557F55890AAA493F551207A19E55793F55212B5AF6038E55700
:20932000B404004008E5520412B5AF6029E55112B5AF6022E558B404004027E5510412B568
:20934000AF6013E558B4061A740212B5AF6007740312B5AF700C90B6031273C31278F6020B
:2093600092D5E551C4F5501278B8E0540FAF82B55848207A10E552C4F5501278B8E0540FCD
:20938000AE82B55735B404004019EF2420F582E0540FB55825207A0BEE2420F582E0540F9B
:2093A000B55717B4061A7802EFF9E92420F9F582E0540FB55804D8F2800690B623029359BC
:2093C0008F509093E11273C312AF0A920C1254CC200C0BD20F12ABBF1278E31278E30292C5
:2093E000D5436D626E2020202020202020202020201264F27876E644FC906800F0E53054CB
:209400000FF558B406028005B40900400D90AAF31273C3D20D43A882805190AAE31273C3AE
:20942000E558C312AEC4F557C312AEC4F556C27C207C1978C97405F6E55712ADFD12AE9ED1
:20944000E55612ADFD74C412AEB5801778C97444F6E55612ADFD12AE9EE55712ADFD74859C
:2094600012AEB5D230753C0043A8A2200D591278D7E53C20E728B41000404C207C14E557C4
:20948000D312AEC440DDF557B5583912966640D38032E556D312AEC440C9F5568026B4F1C2
:2094A000005024207C14E557D312AEE740B5F557B5581112967840AB800AE556D312AEE729
:2094C00040A1F556029430E53890680070207538147876E644FCF4600FF4F550E0B5500B94
:2094E00075380830E04B804D7550FFE550F01264F2202B0302946B127A02500712ADCF5329
:20950000210F2208200D18E6541C601320E42E20E305207C258003307C20B27C029430089D
:20952000E6541F70D708E65403600F75381430E0040559800215590291E802946B53A8DD60
:20954000C230E558B5570B90B6131273C31278F680AA90AAA493F551E55793F552E55693DF
:20956000F553E55112B5AF6025E558B404004008E5510412B5AF6016E55212B5AF600FE50E
:2095800057B404004014E5520412B5AF700C90B6031273C31278F60294FCE551C4F5501247
:2095A00078B8E0540FAE82B5582DE552C4F5501278B8E0540FAC82B5571DB40400401EEEAE
:2095C0002420F582E0540FB5580DEC2420F582E0540FB55702800690B623029591909656E8
:2095E0001273C312B2917F0012B31B885AE558B40400401005510552055312B2917F10124D
:20960000B31B885BD20F12ABBF1278E31278E3C059855630123C0C752F0F12530BAF5A7E3A
:20962000007D617B0A12AD9FE558B404004009AF5B7E107B0A12AD9FE53090AAA493FE121A
:20964000B5A3E530B404004005EE0412B5A31258E1D0590294FC4D69782020202020202030
:20966000202020202020E558B404005003B403041557D3220557C322E558B40400500270CE
:20968000040557D3221557C3221264F27876E644FC906800F0E530540FF558B406028005BA
:2096A000B40900400D90AB131273C3D20D43A882800890AB031273C3C27C200D1DE558C328
:2096C00012AEC4F55778C97443F6E55712ADFD12AE9ED230753C0043A8A2200D3A1278D76E
:2096E000E53C20E719B41000402DE557D312AEC440E0F557B558D312966640D680CCB4F104
:20970000005014E557D312AEE740C7F557B558BA12967840BD80B3E5389068007020753873
:20972000147876E644FCF4600FF4F550E0B5500B75380830E04080427550FFE550F012644F
:20974000F2302B96127A025016800C200D09207C06855730123C0C12ADCF53210FC322086A
:20976000E620E41B08E6541F70ED08E6540360A775381430E0040559800215590291E8201C
:209780000D9553A8DDC230E558B5570E90B6131273C31278F6D27C02974B90AAA493F551FC
:2097A000E55793F552E55112B5AF6028E558B404004008E5510412B5AF6019307C1BE552FB
:2097C00012B5AF600FE557B40400403EE5520412B5AF703690B60380B6E55212B5A3909893
:2097E000721273C312B32DE558B40400400C05510552E55212B5A312B32DD20F12ABBF12CD
:2098000078E31278E3C20D02974BE551C4F5501278B8E0540FB5582FAE82E552C4F550124B
:2098200078B8E0540FB5571FAC82B40400401EEE2420F582E0540FB5580DEC2420F582E0B9
:20984000540FB55702800690B62302978F9098821273C312B436E558B404004007055105FB
:209860005212B436D20F12ABBF1278E31278E3029757436F70792020202020202020202098
:209880002020537761702020202020202020202020201264F27876E644FC906800F0E530F4
:2098A000540FF558B406028005B40900400D90AB331273C3D20D43A882800890AB23127340
:2098C000C3D27C0296BA1264F27876E644FC906800F043A88290AB431273C3E53890680079
:2098E00070207538147876E644FCF4600FF4F550E0B5500B75380830E03180337550FFE525
:2099000050F01264F2302BD3127A02500712ADCF53210F2208E620E41B08E6541F70EE0885
:20992000E6540360B675381430E0040559800215590291E8E530540FF55890AAA493F551BA
:2099400012B5AF6029E558B40400402EE5510412B5AF601AE558B406028005B40900401AE6
:20996000740212B5AF6007740312B5AF700C90B6031273C31278F602990D909B9E1273C361
:20998000755600E55890998B93800B00010203040506000204002556F557E556C4F55012B5
:2099A00078B8C2E704F582E0540FF0A3A3A3E0A3F55BE0F55CE5822409F582E0C4540C0321
:2099C00003F55AC083C082E5572323FF0F909BAE93F55DEF0F93F55EEF93F55F1268A58504
:2099E0005A5D855B5E855C5FEF1F909BCA93F55CEF1F93F55BEF93F55A1268A5D082D083C5
:209A0000E58224FEF582E55BF0A3E55CF0E5822402F582E0540FC55AC4455AF0E58224F905
:209A2000F582E0F55EA3E0F55FE5822405F582E0A3C4540C0303F55DC083C082E557232398
:209A4000FF0F909BCA93F55AEF0F93F55BEF93F55C1268A5EF1F909BAE93F55FEF1F93F5EA
:209A60005EEF93F55D126892D082D083E05430C4FF1582E054304FFFE55DC423234FF0E523
:209A80008224F6F582E55BF0A3E55CF0A37F02E4F0A37404F0A3A3A3DFF515821582E0FFE2
:209AA000A3E0FEE58224FBF582EFF0A3EEF0E5572323FF0F909BAE93F8EF0F93F9EF93FACE
:209AC000EF1F909BCA93FDEF1F93FCEF93FBE8C4FEE9C4540F4EF8E944F0F9EBC4FEECC466
:209AE000540F4EFBEC44F0FCC20F12ABBF90E008E8F089838A82E090E004E0A3F55AE0F5EE
:209B00005B90E008EBF08C838D82E090E004E0A3F55CE0F55D90E004E55AF0A3E55BF09019
:209B2000E008E8F089838A82F090E004E55CF0A3E55DF0755A00895B8A5C12693D435BF004
:209B4000A95BAA5C30780808C20FD27E12ABBF755A008C5B8D5C12695C435BF0AC5BAD5C92
:209B60003078011BE88B5AB55A005003029AEDE558B4070040140556B40A00E5565008B4BD
:209B800002028006029983B404FA1258E1D20F12ABBF1278E31278E375590402990D5276A7
:209BA000727320202020202020202020202001000000018000000200000002800000010039
:209BC00000000200000001000000017FFFFF01FFFFFF027FFFFF02FFFFFF01FFFFFF02FF89
:209BE000FFFF02FFFFFF1264F27876E644FC906800F0906191740DF090AB531273C378C9FA
:209C00007445F6906484E0A2E39278A2E2E492E0A27892E1909CD193C23053A8DD909CD5EC
:209C2000F55F93FF906484E054F34FF0E55F042430906190F012AEABD230753C0043A8A2A8
:209C40001278D7E53C20E70FB410004017E55F04B4040050E380C1B4F1005008E55F142068
:209C6000E7D680B4E53890680070207538147876E644FCF4600FF4F550E0B5500B75380838
:209C800030E03780397550FFE550F01264F2302BAF127A02500A75590512ADCF53210F227B
:209CA00008E654106002803108E6541F70E808E65403600F75381430E004055980021559AF
:209CC0000291E8029C4090B6031273C31278F680C50100030204000C0853A8DDC230755D1B
:209CE00000E530540FF55812CF5740AA12B5B9F5F0909D3A1273C3532FF3E5F0128DFCE59F
:209D000030540FB4070050111258E1D20F12ABBF1278E31278E3029C96055DE5F004128D04
:209D2000FCE530540FB40AE0755D027402128DFC755D037403128DFC80CE4C6F6F7020201D
:209D40002020202020202020202090AB631273C3532F00755764803190AB731273C3532F02
:209D600000432F80755701802090AB831273C3532F00432F40755764800F90AB931273C375
:209D8000532F00432FC07557011264F27876E644FC906800F0755600E530540FF55890605E
:209DA00001E013927A5006307F03755702C23053A8DD307D03029DF478C97406F6E55712C1
:209DC000A920906190781FE618F0A3B46BF9740DF012AEABE55612A93D75A080780074C5A4
:209DE000F2087A03791FE719F208DAFA123AFB1278ED804CE55712A92075A08078007486DE
:209E0000F208EFF208EEF208123AFB1278ED780074C0F208791DE719F208B46BF9123AFB24
:209E20001278ED78C97445F6E55612A93D906190781F7A03E618F0A3DA8D740DF012AEAB1F
:209E4000D230753C0043A8A21278D7E53C20E728B404004041207D12E55704307A0104B486
:209E60006500400280DAF557800B24FD255630E70280CDF556029DADB4FD005019207D10AA
:209E8000E55714307A0614B4020040B470D180B02403255680D8E538906800702075381433
:209EA0007876E644FCF4600FF4F550E0B5500B75380830E04580477550FFE550F01264F2E0
:209EC000302B85127A02500712ADCF53210F2208E6541C601320E42E20E305207D2580033A
:209EE000307D20B27D029DAD08E6541F70DA08E65403600F75381430E00405598002155998
:209F00000291E8029E4853A8DDC230E55890AAA493F55112B5AF700C90B6031273C3127813
:209F2000F6029EC8E551C4F5501278B8E0540FB55835B407004036E5510412B5AF60D9E5BE
:209F4000822420F582E0540FB5581CB4091FE52144F0F470C37F02E5822420F582E0540F35
:209F6000B55804DFF2800690B623029F1B207E0B90A4C9307F0E90A4D9800990A4E9307F8F
:209F80000390A4F91273C3C20F12ABBFC050C056C057755732D27A12A765D057D056D050EA
:209FA000E5571423F55790B63E93F509F55CF55EE5570493F508F55DF55F12A956F50B851D
:209FC0005D0AE55623F55690B70693F50DF55CE5560493F50CF55D85095E85085F12A95630
:209FE000F50F855D0EE50E250AF55FE50F350B2420F55EE4755A04F55BF55CF55D12AA4F77
:20A00000F507855C06207F15855C5DF55C850B5E850A5F12A956F501855D008005F5018555
:20A020005C00E4C3950AF55D7420950BC55DC333C55D33F55C85075E85065F12A956F5035D
:20A04000855D02E50EC3950AF55DE50F950BC39420F55C85075E85065F12A956F505855D58
:20A0600004C20F12ABBFE42404F582758360E0F553A3E0F554E5822403F582E0F556A3E00D
:20A08000F557E5822405F582E0F55554C00303F55FE553C4540F455FF552E55344F0F553D7
:20A0A000E5555403C4F555E556C4540F4555F555E55644F0F556E4F50BF50AF50DF50CF526
:20A0C00013F512F515F51485520E85530F85541690E008E50EF0850F83851682E0A385827F
:20A0E00016E5837009C20F12ABBF050E74F0F50F90E004E0F508A3E07F03A2E713C50813CF
:20A10000C508DFF6F509E50AC333F506E50B33F507207F0CE5082506F506E5093507800B2D
:20A12000E508C39506F506E5099507C506250CF55FE506350DF55E85015C85005D12A956AA
:20A14000855D06F50785035C85025D85135E85125F12A956C506255DC5063507F50785057C
:20A160005C85045D85155E85145F12A956307C1AC506255DF55DE5063507F55C857C5E85DB
:20A180007D5F12A956855D10800AC506255DF510E5063507F511F50730E701F454F0700318
:20A1A00002A246E51130E70EE510F42401F55FE511F43400800585105FE511755A01755B0B
:20A1C000FF755CC0755D0012AA4FF57DE55CC333C57D33F57CD27CA852A953AA54EAB5168C
:20A1E00010E9B50F0CE8B50E0885115C85105D808B90E008E8F089838A82E0A3AA82E58375
:20A2000070030874F0F990E004E0F55DA3E07F03A2E713C55D13C55DDFF6F55C857C5E85BE
:20A220007D5F12A9567F03C55D33C55D33C55DDFF830E3082410C55D3400C55D90E004F0E1
:20A24000A3E55DF080977F03E51033C50733C507DFF830E3082410C5073400C50790E00437
:20A26000F0A3E507F0850A0C850B0D85080A85090B851214851315851012851113E516B5AF
:20A28000570CE50FB55607E50EB55502800302A0D0207E0302A492C20F12ABBFE552C555EA
:20A2A000F552E553C556F553E554C557F554E4F50BF50AF50DF50CF513F512F515F514C254
:20A2C0007C85520E85530F85541690E008E50EF0850F83851682E0E516C39401F516E50F86
:20A2E0009400B4EF09C20F12ABBF150E74FFF50F90E004E0F508A3E07F03A2E713C5081365
:20A30000C508DFF6F509E50AC333F506E50B33F507207F0CE5082506F506E5093507800B2B
:20A32000E508C39506F506E5099507C506250CF55FE506350DF55E85015C85005D12A956A8
:20A34000855D06F50785035C85025D85135E85125F12A956C506255DC5063507F50785057A
:20A360005C85045D85155E85145F12A956307C1AC506255DF55DE5063507F55C857C5E85D9
:20A380007D5F12A956855D10800AC506255DF510E5063507F511F50730E701F454F0700316
:20A3A00002A447E51130E710E510F42401F55FE511F43400F55E800685105F85115E755A83
:20A3C00001755BFF755CC0755D0012AA4FF57C855C7DD27CA852A953AA54EAB51610E9B5CB
:20A3E0000F0CE8B50E0885115C85105D808E90E008E8F089838A82E0EAC39401FAE994009C
:20A40000B4EF031874FFF990E004E0F55DA3E07F03A2E713C55D13C55DDFF6F55C857C5EEF
:20A42000857D5F12A9567F03C55D33C55D33C55DDFF830E3082410C55D3400C55D90E0044A
:20A44000F0A3E55DF080937F03E51033C50733C507DFF830E3082410C5073400C50790E04D
:20A4600004F0A3E507F0850A0C850B0D85080A85090B851214851315851012851113E5165E
:20A48000B5570CE50FB55607E50EB55502800302A2CAE530540F207B0EB407004013055129
:20A4A000D27B742002A067B40A070551E551B4040ED20F12ABBF1278E31278E3029EC8C438
:20A4C000F5501278B8C2E780DB4C50463120202020202020202020202048504631202020EF
:20A4E0002020202020202020204C5046322020202020202020202020204850463220202038
:20A50000202020202020202020171F272F1F2F2F17271F171264F27876E644FD906800F039
:20A5200090ABA31273C378C97444F6E530540FF558755732C23053A8DD906190E55775F057
:20A5400064842430F0A3E5F075F00A842430F0A3E5F02430F0A3740DF012AEABD230753C32
:20A560000043A8A21278D7E53C20E713B40500401924FC2557B4650050E4F55702A534B4DC
:20A58000FC0050062404255780EBE538906800701D7538147876E644FDF4600CF4F550E069
:20A5A000753808B55005803A7550FFE550F01264F27874E6540C700612A68902A534302BB2
:20A5C000A3127A02500712ADCF53210F2208E620E41808E6541F70EE78C6E65402753814BC
:20A5E000600515590291E802A56453A8DDC230E55890AAA493F55112B5AF700C90B60312F7
:20A6000073C31278F602A5C6E551C4F5501278B8E0540FB55844B404004045E5510412B5C4
:20A62000AF60D9E5822420F582E0540FB5582BB406028005B409004027E52144F0F470BCD6
:20A64000E5822420F582E0540FB5580EE5822420F582E0540FB55802800690B62302A5FF71
:20A6600090A6791273C3C27A12A765D20F12ABBF1278E31278E302A5C64C65766C202020F2
:20A6800020202020202020202053A8DDC23090A73F1273C3E530540F23F55290A74F93C552
:20A6A000520493F555E4F554F55774F0F553F55685520E85530F855416755E00755F009005
:20A6C000E008E50EF0850F83851682E0A3858216E5837004050E74F0F50F90E004E0F55BE0
:20A6E000A3E030E70AC55BF42401C55BF43400F55AB55E07E55BB55F0280084006855A5E6B
:20A70000855B5FE516B5570CE50FB55607E50EB55502800302A6BFE4F55A855E5B855F5C47
:20A72000F55D755E8004F55F12AA4FE55C75F064A433E5F03400F55790ABA31273C3222073
:20A740005365656B204D6178206C6576656C201018182020282830102020301030102020C3
:20A76000301030103085575C755D00755E28755FF012A9F1C57B548023255EF57DE57B34F4
:20A7800000F57C532FFC755004758360855082E0F553A3E0F554E5822403F582E0F556A38B
:20A7A000E0F557E5822405F582E0F55554C00303F55FE553C4540F455FF552E55344F0F523
:20A7C00053E5555403C4F555E556C4540F4555F555E55644F0F55685520E85530F855416CC
:20A7E000207A07D27EC20F12ABBF755E00755F0090E008E50EF0850F83851682E0A385825B
:20A8000016E583700C207A05C20F12ABBF050E74F0F50F90E004E0F55BA3E030E70AC55B6F
:20A82000F42401C55BF43400F55AB55E07E55BB55F0280084006855A5E855B5FE516B557A7
:20A840000CE50FB55607E50EB55502800302A7F0E55E7F03A2E713C55F13C55FDFF6755A6B
:20A8600000857C5B857D5C755D0030E706F4C55FF4C55FF55E12AA4FF50E855C0F207A050F
:20A88000C20F12ABBF90E008E552F0855383855482E0A3858254E583700C207A05C20F12D2
:20A8A000ABBF055274F0F55390E004E0F55DA3E07F03A2E713C55D13C55DDFF6F55C850ED4
:20A8C0005E850F5F12A9F17F03E57B33C55E33C55EDFF890E004F0A3E55EF0E554B5570C8B
:20A8E000E553B55607E552B55502800302A88520780FE558B407004016755024D27802A748
:20A9000089E558B40A09E5502420F550B484EF224C65766C20202020202020202020202090
:20A920007D307C6B307A010375F00A84B40A057F207E31222DFF7E2EE5F0421D227F307E54
:20A94000307D3075F06484421FE5F075F00A84421EE5F0421D22E55EC2D530E70EB2D5F474
:20A96000C55FF42401C55F3400F55EE55C30E70EB2D5F4C55DF42401C55D3400F55CE55FE8
:20A98000855DF0A4E55EC5F0C55DA4255DF55DE435F0F57BE433C55F855CF0A4255DC57BC4
:20A9A00035F0C55F3400C55E855CF0A4255FC55E35F0F55FE57B33C55E33C55F33C55E33CC
:20A9C000C55F33C55E33C55F33C55E33C55F3330D511F4C55FF4C55EF42401C55E3400C54C
:20A9E0005F3400F55DE55E33E55F3400C55D340022C2D5E55C30E70EB2D5F4C55DF4240159
:20AA0000C55D3400F55CE55F855DF0A4E55EC5F0C55DA4255DF55DE435F0F57BE433C55F8F
:20AA2000855CF0A4255DC57B35F0C55F3400C55E855CF0A4255FC55E35F030D511F4C55ED1
:20AA4000F4C57BF42401C57B3400C55E3400227F10E55BC3955FE55A955EB34046D3E55DB6
:20AA600033F55DE55C33F55CE55B33F55BE55A33F55A92D5E55BC3955FF55BE55A955EF533
:20AA80005A20D511500FE55B255FF55BE55A355EF55A535DFEDFC6E55A33E55D3400C55C66
:20AAA0003400C322000102030002000002000001030301202057617665206D6F64696679F0
:20AAC0002020202020436F6D62696E6520202020202020436F6D62696E652073747220657E
:20AAE000727220204D697820202020203D3E2020202020204D6978207374722020657272F9
:20AB00006F72202020436F707920203D3E202020202020436F707920737472202065727241
:20AB20006F7220202053776170203C3D3E2020202020205377617020737472202065727205
:20AB40006F7220202020205265766572736520202020204C6F6F702020204D6F6465202039
:20AB60003120204C503120463D2020202020523D20202048503120463D2020202020523DCA
:20AB80002020204C503220463D2020202020523D20202048503220463D2020202020523DB9
:20ABA0002020204C766C2041646A204D61783D20202025AAC3AAE3AB03AB23AB43AB53303E
:20ABC0000E0122C083C082C0E090610FE004F0906190E4F0A3740DF0E530540F90ABE493B8
:20ABE00090ABEF73000000000A0A130A0A1313207E0A90610FE023801C207E0990610FE089
:20AC00008013207E0890610FE0C313800890610FE054FC0303602FB40300500474018026D2
:20AC2000B4050050047402801DB40600500474038014B4080050047404800BB40A005004B6
:20AC40007405800224FC53A8C1C230B40C004004D20E740C90AC5C9390AC697300050A0F66
:20AC600014191E23282D32373790ACF7803590AD05803090AD13802B90AD21802690AD2F2C
:20AC8000802190AD3D801C90AD4B801790AD59801290AD67800D90AD75800890AD83800308
:20ACA00090AD91C018C01F75A08078007484F208C3123AE0123AFB1278ED780074C0F208BD
:20ACC000C3123AE01278EDE49378C9F612AEAB43A882D230908080740FF08568A0D01FD037
:20ACE00018D0E0D082D083300F0C200E091278E31278E302ABBF22002020200D2020202010
:20AD000020202020042D0020200D2020202020202020052D2D00200D2020202020202020A9
:20AD2000062D2D2D000D2020202020202020072D2D2D2D0D0020202020202020402D2D2D0A
:20AD40002D0D2D00202020202020412D2D2D2D0D2D2D002020202020422D2D2D2D0D2D2D73
:20AD60002D0020202020432D2D2D2D0D2D2D2D2D00202020442D2D2D2D0D2D2D2D2D2D0028
:20AD80002020452D2D2D2D0D2D2D2D2D2D2D0020462D2D2D2D0D2D2D2D2D2D2D2D00478D29
:20ADA000838F82E0A3AF828D838E82F0A3AE82DBEE228D838F82E0C0E08E82E0FCD0E0F050
:20ADC000A3AE828D838F82ECF0A3AF82DBE42253A8C1C230906484E0C454F04559C4F07519
:20ADE000A08090FF927B017440123B067870790774FFF608D9FC908080740FF022540F2336
:20AE0000F55090AE1293F551E5500493F58285518322AE2AAE2EAE32AE36AE3AAE3EAE42CA
:20AE2000AE47AE4BAE4FAE55AE5D4120200D4220200D4320200D4420200D4142200D4344A4
:20AE4000200D414243440D412F420D432F440D41422F43440D412F422F432F440D2A2020D8
:20AE60000D1264F2202B051278D380F5127A025012906484E0C454F84559C4F053A8FDC2D7
:20AE800030D32278C4E630E2040559800A30E3D1155930E70224FC53A8FDC230C32275A0FE
:20AEA000617890E493A3F208B40DF878C77466F6087401F62275A0807800F208C3123AE0C2
:20AEC000123AFB22400590AEDD9322B403028008B405028003B40802D322C380E701020392
:20AEE00000050406080709400590AF009322B400028008B404028003B40702D322C380E79B
:20AF000003000102050406080709755400E558B4040050065401C403F554E558B40610750F
:20AF200051107552F075530075828E7440801EE550240EF582758360E0030354304554F52C
:20AF4000517552F0755300E551232354C0C082906FFFF0532FFCD0E024F6F582758360E06A
:20AF6000F55E207804E554C4F0A3E0F55D207802E4F0E5822403F582E0F55BA3E0F55A307B
:20AF80007A3CE55D7038E55E547F7032D279E558B40400400CB406028024747FB55B00501A
:20AFA0001D90AFAEC2A91273C31278F6D3224E6F206E65656420746F20436F6D626EE5826D
:20AFC0002405F582E0F55C03035430F55FE55EC4540F455FF55FE55E44F0F55EE55C5403FE
:20AFE000C4F55CE55BC4540F455CF55CE55B44F0F55BC20F12ABBF30790FE558B4060A74A5
:20B000001FB55C00500302AFA1307A0302B0B930780302B07590E008E55CF0855B83855A86
:20B0200082E090E005E033927F7801E55AC398F582E55B9400F583B4F000500EC08290E08B
:20B0400008E55C14F0D0827583F0E090E005E033207F08400808E8600480D040F8927FE540
:20B060005AC398F55AE55B9400F55BB4F0005002155C02B0B990E008E55FF0855E83855DE2
:20B0800082E090E405E033927E780190E405E033207E08400808E8600F80F040F8207F0613
:20B0A0004006927E80EF40FAE55D28F55DE55E34007004055F74F0F55E90E008E55FF0859E
:20B0C0005E83855D82E0A385825DE5837009C20F12ABBF055F74F0F55E90E004E0FDA3E027
:20B0E000FC90E008E551F0855283855382F0A3858253E5837004055174F0F55290E004EDD7
:20B10000F0A3ECF0E55DB55A0CE55EB55B07E55FB55C02800302B0B9207A0B207808EE246D
:20B1200004D27802AF5A90B12EE558938007171F272F1F2F1FB55100501190B144E558933B
:20B14000F530802E04000500060006E558B406027404F530B404004019B4050C7427B551FA
:20B1600000400F753002800A7417B551004003753000907A10E55893C4F45521F521E5576C
:20B1800093C4F45521F521E53093C44521F521207A54E5502406CE2406FF7D607B0212AD93
:20B1A0009FEF2402FFEE2402FE7B0212AD9FEECFFE2402F582E0540CC0E0EF2402F582E04B
:20B1C00054F3F8D0E048F0EE2404F582E054CFC0E0EF2404F582E05430F8D0E048F0EF2433
:20B1E000F4FFEE24F4FEE5515430C4C551540FC4C552540F4552F552E553C39401F553E588
:20B20000529400F552E5519400F551E5502408F582758360E552F0A3E553F0E5822403F54C
:20B2200082E552F0A3E553F0A3C082906FFFE0F508758360D082E0543C45084551F0A3E06A
:20B2400054CFC44551C4F05382F0E054F04530F0540FB404004038EF2420FEF582E054F010
:20B260004530F00F0E7D607B1F12AD9FE530B4061E7582C07426F07582E07436F07F817E5A
:20B28000C17B1F12AD9F7F817EE17B1F12AD9FC322E551C4F5501278C5F55FE552C4F55097
:20B2A0001278C5F55EE553C4F5501278C5F55D755B007B08755CF0C20F12ABBF90E008E54C
:20B2C0005FF0855C83855B82E090E004E0FFA3E0A2E713CF13FE90E008E55EF0855C838593
:20B2E0005B82E0A385835C85825B90E004E0FDA3E0A2E713CD132ECD3FFE90E008E55DF0F6
:20B3000090E004EDF0A3EEF0E55C600302B2BC055F055E055DDB012202B2B4E553C4F55077
:20B320001278ACFEF87D617B0A12AD9F22E551C4F5501278B804FFE552C4F5501278B8E513
:20B3400057C44552C4F0A3AE82AD837B0312AD9F8F82E0F8A3AF82E55712B5C08E82F0A385
:20B36000AE827B0112AD9F7A027B0212AD9F8F82E0F8A3AF82E55712B5E38E82F0A3AE82F6
:20B380007B0112AD9FDAE28F82E0C0E0A3AF82E55790B63393FBD0E0543C4B8D838E82F0D4
:20B3A000A3AE828F82E0C0E0A3AF82EB5403C4FBD0E054CF4B8E82F0A3AE827B1012AD9F7A
:20B3C000E551C4F5501278ACFFE552C4F5501278ACFE7D617B0A12AD9FE551C4F5501278FB
:20B3E000C5F55FE552C4F5501278C5F55E7908755C00755DF0C20F12ABBF90E008E55FF045
:20B40000855D83855C82E0A385835D85825C90E004E0F55BA3E0F55A90E008E55EF090E088
:20B4200004E55BF0A3E55AF0E55D70CE055F055ED9012202B3F2E551C4F5501278B804FF98
:20B44000E552C4F5501278B804FE7D607B0312ADB28F82E0F8E55712B5C0C0E08E82E0F868
:20B46000E55812B5C0FCD0E0F0A3AE828F82ECF0A3AF827B0112ADB27A027B0212ADB28FF2
:20B4800082E0F8E55712B5E3C0E08E82E0F8E55812B5E3FCD0E0F0A3AE828F82ECF0A3AF4F
:20B4A000827B0112ADB2DAD28F82E0C0E0E55790B63393FBD0E0543C4BC0E08D838E82E072
:20B4C000FCE55890B63393FAEC543C4AFCD0E08D838E82F0A3AE828F82ECF0A3AF82E0C077
:20B4E000E0EB5403C4FBD0E054CF4BFB8E82E0C0E0EA5403C4FAD0E054CF4AFAEBF0A3AE80
:20B50000828F82EAF0A3AF827B1012ADB2E551C4F5501278ACFFE552C4F5501278ACFE7D89
:20B52000617B0A12ADB2E551C4F5501278C5F55FE552C4F5501278C5F55E7908755C007529
:20B540005DF0C20F12ABBF90E008E55FF0855D83855C82E090E004E0F55BA3E0F55A90E017
:20B5600008E55EF0855D83855C82E0A385835D85825C90E004E0FFA3E0FE90E004E55BF005
:20B58000A3E55AF090E008E55FF090E004EFF0A3EEF0E55D600302B547055F055ED90122F3
:20B5A00002B53F04FFD3E433DFFD4521F5212204FFD3E433DFFD552122908B4EE558932272
:20B5C000B404005010B401028003B40304E8448022E8547F22B406005002E822E552134013
:20B5E000EC80EEB40400500D6003B40204E8547F22E8448022B406005002E822E552135064
:20B60000EC80EE5761726E2020456D7074792062616E6B5761726E20202053616D6520622D
:20B62000616E6B2053747220206D6973736D6174636820414182824182824182000000566A
:20B6400000AC0101015701AD0203025A02B00306035D03B4040B046204BA0511056A05C284
:20B66000061B067406CD0727078107DC0837089308EF094C09A90A070A660AC50B250B85DB
:20B680000BE70C490CAB0D0F0D740DD90E3F0EA70F0F0F780FE3104E10BB1129119812086A
:20B6A000127A12ED136113D7144F14C8154315BF163E16BE174017C4184A18D2195D19EA17
:20B6C0001A791B0B1B9F1C361CD01D6D1E0D1EB01F56200020AD215F221422CD238A244C12
:20B6E000251325DE26AE2784286029412A292B172C0B2D072E0B2F16302A3147326D339CE0
:20B7000034D7361C376D30002F4F2E9F2DF02D432C982BED2B442A9D29F7295228AE280C69
:20B72000276C26CC262E259224F7245D23C4232D22982203217120DF204F1FC01F331EA7D1
:20B740001E1C1D931D0B1C851C001B7C1AFA1A7919F9197B18FE188318091790171916A3D4
:20B76000162E15BB154914D9146A13FC1390132512BC125411ED1188112410C110601000B1
:20B780000FA20F450EE90E8F0E360DDE0D880D330CE00C8E0C3D0BEE0BA00B530B080ABE60
:20B7A0000A760A2F09EA09A50962092108E108A20865082907EE07B5077D0747071206DEE9
:20B7C00006AC067B064C061D05F105C5059B0573054B0525050104DE04BC049C047D045F43
:20B7E00004430428040F03F703E003CB03B703A40393038303750368035C03520349034174
:20B80000033B033703330004021F020400000004081F0804000090CFFAE530540FF5589367
:20B82000C4F5501278B8F55FE0758200F0E558B407004023B4090474C08004E55F2420F551
:20B8400082E0758220F0E558B40A0C906040742AF0906060743AF075D01875381075A0801D
:20B8600090B8067B027440123B06C299D29C43A8921264F27876E644FC906800F0E4F52F44
:20B88000F55F90D1601273C3803175D0187401F52FF55F90D1701273C3802075D018752F96
:20B8A00000755F0290D1801273C3800F75D018752F01755F0390D1901273C3E500B5016BE2
:20B8C000E53890680070207538107876E644FCF4600FF4F550E0B5500B75380830E03080F1
:20B8E000367550FFE550F01264F2302BCE127A025007D27AD27F02D10B08E6541060030281
:20B90000B9C578C6E6540360B275381020E108E55F04B4040880A4E55F1420E79E90B925BF
:20B920009390B8577300334455809012D00540F9B44107755F01D278802DB4122212D04193
:20B94000B40202800DB406028008B40A028003B40ED718755F02C278D27975D0188066B418
:20B96000405A755F03D27812D041B40202800DB406028008B40A028003B40EADF55E12D079
:20B9800041703F12D041703A12D041B411005032F55D12D041702B12D0417026E55D255EF2
:20B9A000F55C12D041255CC2E7701712D04130E711E55FB4010302C5B002CA3F75D018023A
:20B9C000B8BB02D10B12CE92E55FC2E003600302BF1712CF575006432FC002D10B90D1A0E1
:20B9E0001273C378C97447F6906190E4F0A3740DF012AEABD23012D04DE55823FF90BA83DC
:20BA000093CF0493F5828F83E493A3307808F309C5F025F0C5F0F55A540CF552540423C529
:20BA20005254087002740423234552F552E43078067F02F309DFFC93307808F309C5F02547
:20BA4000F0C5F0232552F55530785C7F02E4F309DFFC12D0F875D018E500B501101264F2D3
:20BA6000302BF5127A0250F0D27A02D10B12D00540E3B443028030B44E0302B9F6B44FD53D
:20BA800002D12ABA99BA9BBA9DBA9FBAA1BAA3BAA5BAA1BAA3BAA5BAA5020406040A040E98
:20BAA0000402080A0802107553F0E4F554F55BF55C85525D85535E85545F12D085E55AF393
:20BAC0000925F0F5F0E55BF30925F0F5F0E55CF30925F0F5F07F4090E008E552F08553833D
:20BAE000855482E0A3858254E583700474F00552F55390E004E0A3FEE0C31392D5F30925FB
:20BB0000F0F5F0A2D5EE13C313F30925F0F5F0E555B55204D27C8002DFBD12D0F875D01824
:20BB200030784AE500B501101264F2302BF5127A0250F0D27A02D10B12D00540E0B44318A2
:20BB4000207C43E55B3401A2E7C2E7F55BE55A3400C2E7F55A02BAB1B44E0C855D52855E12
:20BB600053855F5402BABAB44FB302D12A302EFD7F001264F2302B0A127A025005D27A0239
:20BB8000D10BDFEE80BA30783012D0BD75D018E500B501101264F2302BF5127A0250F0D2EB
:20BBA0007A02D10B12D00540E3B44302800BB44E0280D3B44FD602D12A12D04DE55823FFE4
:20BBC00090BDD993CF0493F5828F833078067401F309F5F0E493A3F55B30784AF30925F04C
:20BBE000F5F07F02E4F309DFFC7F02E493A3F30925F0F5F0DFF512D0F875D018E500B501ED
:20BC0000101264F2302BF5127A0250F0D27A02D10B12D00540E3B44302800BB44E028099B9
:20BC2000B44FD602D12A12D0857401F309F5F0E55BF30925F0F5F0E4F3099061007F09E002
:20BC4000A3F30925F0F5F0DFF69060007F20E0A3FE540FF30925F0F5F0EEC4540FF30925D7
:20BC6000F0F5F0DFE9E558B40700500302BC9A9061107F09E0A3F30925F0F5F0DFF69060BD
:20BC8000207F20E0A3FE540FF30925F0F5F0EEC4540FF30925F0F5F0DFE912D0F875D01801
:20BCA00030782BE500B501101264F2302BF5127A0250F0D27A02D10B12D00540E0B4430256
:20BCC0008023B44E0302BC26B44FD202D12A302EFD7FAB1264F2302B0A127A025005D27A85
:20BCE00002D10BDFEEE558B40A02800920780302BE1002BDA912D0857401F309E4F3097414
:20BD000052F30975F0539061207F09E0A3F30925F0F5F0DFF69060407F20E0A3FE540FF390
:20BD20000925F0F5F0EEC4540FF30925F0F5F0DFE99061307F09E0A3F30925F0F5F0DFF636
:20BD40009060607F20E0A3FE540FF30925F0F5F0EEC4540FF30925F0F5F0DFE912D0F875F8
:20BD6000D01830782BE500B501101264F2302BF5127A0250F0D27A02D10B12D00540E0B4F2
:20BD800043028025B44E0302BCF5B44FD202D12A302EFD7FAB1264F2302B0A127A025005FA
:20BDA000D27A02D10BDFEE806712D0BD75D018E500B501101264F2302BF5127A0250F0D2A6
:20BDC0007A02D10B12D00540E3B443028042B44E0280D6B44FD602D12ABDEFBDEFBDEFBD55
:20BDE000EFBDEFBDEFBDEFBDF2BDF2BDF2BDF5000049000112000224BE00BE04BE08BE0CFF
:20BE00001820303020303030283030303030303012D04D3078467401F3097408F3097F03DA
:20BE2000E4F309DFFC7428F30975F03112D0F875D018E500B501101264F2302BF5127A02F1
:20BE400050F0D27A02D10B12D00540E3B44302800BB44E0280BAB44FD602D12A12D08574FB
:20BE600001F3097408F309E4F30975F0099064007F14E0A3FE540FF30925F0F5F0EEC45498
:20BE80000FF30925F0F5F0DFE912D0F875D01830782BE500B501101264F2302BF5127A02DA
:20BEA00050F0D27A02D10B12D00540E0B443028022B44E0302BE5CB44FD202D12A75D01826
:20BEC000302EFDC23075A08090FF927B027440123B062212D0BD75D018E500B5011012649C
:20BEE000F2302BF5127A0250F0D27A02D10B12D00540E3B4431675D018302EFDC23075A032
:20BF00008090FF927B027440123B0622B44E0280DAB44FC202D12A3079097568658568A039
:20BF200002BFB390D1C01273C330785312D069E55823FF90BA8393CF0493F5828F83E493B9
:20BF4000A3F309C5F025F0C5F0F55A540CF552540423C55254087002740423234552F552D1
:20BF6000E47F02F309DFFC93F309C5F025F0C5F0232552F5557F02E4F309DFFC12D0F87508
:20BF8000D018E500B501101264F2302BF5127A0250F0D27A02D10B12D00540E3307811B4E7
:20BFA00042028036B44E0302BF17B44FD202D12AB412CC12D041B40F0050C4F55AF5F01206
:20BFC000D04170BB12D04170B675D018E55A540C0303C4F5501278C5F55275D01890D1B0CD
:20BFE0001273C378C97447F69061907401F0A3740DF012AEABD2307568658568A07553F019
:20C00000E4F554F556F55BF55C20784202C09075D018E500B501101264F2302BF5127A028D
:20C0200050F0D27A02D10B12D00540E330781CB44202801AB44F0302D12AB445D212D0A3E3
:20C0400002C1282078DE150002C128B412C1E556C2E7255CA2E7C2E7F55CE55654802335A9
:20C060005BA2E7C2E7F55BE55A3400C2E7F55A75F00012D041B55ACB25F0F5F012D041B544
:20C080005BC125F0F5F012D041B55CB725F0F5F075560085525D85535E85545F90E008E5DB
:20C0A00052F0855383855482F0A3858254E583700474F00552F55312D041FE12D04120E770
:20C0C0002005560556C5F025F0C5F0233392D590E004F0A3EEC5F025F0C5F0A2D533F080C0
:20C0E000BBE5F02EC2E77026E554C39401F554E553540F940044F0F553E5529400F552129A
:20C10000D0A330780302C00F207C1D02C00F20780302D12A12D0DE855D52855E53855F54AC
:20C12000755600C27C02C00F20780302C1A112D069E55823FF90BDD993CF0493F5828F83D4
:20C140007401F309F5F0E493A3F55BF30925F0F5F07F02E4F309DFFC7F02E493A3F3092531
:20C16000F0F5F0DFF512D0F875D018E500B501101264F2302BF5127A0250F0D27A02D10B84
:20C1800012D00540E3307816B442028033B44F0302D12AB445D212D0A3C27D02C348B412C7
:20C1A000C775F00012D041B401D325F0F5F012D04125F0F5F012D04170C325F0F5F08020A1
:20C1C00075F00012D041B401B425F0F5F012D041B55BAA25F0F5F012D04170A125F0F5F06F
:20C1E0009061007F0912D041F0A325F0F5F0DFF59060007F2012D041FE25F0F5F012D04175
:20C20000C5F025F0C5F0C44EF0A3DFE912D041FE12D04130E70302C25D906110CEF0A3252C
:20C22000F0F5F0EEF0A325F0F5F07F0712D041F0A325F0F5F0DFF59060207F2012D041FED4
:20C2400025F0F5F012D041C5F025F0C5F0C44EF0A3DFE912D041FE12D04130E707EE25F070
:20C26000C2E7600C20780302D12A12D0DE02C16812D0A375D018E500B501101264F2302BD6
:20C28000F5127A0250F0D27A02D10B12D00540E3307816B442028014B44F0302D12AB44561
:20C2A000D212D0A3C27D02C348B412C712D041B401D612D041B40805D27D02C34870C91215
:20C2C000D041B452C375F0539061207F0912D041F0A325F0F5F0DFF59060407F2012D041BD
:20C2E000FE25F0F5F012D041C5F025F0C5F0C44EF0A3DFE99061307F0912D041F0A325F0C3
:20C30000F5F0DFF59060607F2012D041FE25F0F5F012D041C5F025F0C5F0C44EF0A3DFE94B
:20C3200012D041FE12D04130E707EE25F0C2E7600C20780302D12A12D0DE02C16812D0A37B
:20C34000C27D30780302C273207D6230781C12D0697401F3097408F3097F03E4F309DFFC88
:20C360007428F30975F03112D0F875D018E500B501101264F2302BF5127A0250F0D27A02D9
:20C38000D10B12D00540E3307814B442028012B44F0302D12AB445D212D0A302C3F8B4129B
:20C3A000C912D041B401D812D041B408D212D04170CD75F0099064007F1412D041FE25F0C8
:20C3C000F5F012D041C5F025F0C5F0C44EF0A3DFE912D04125F0C2E7600F12D0412078035B
:20C3E00002D12A12D0DE02C36A12D04130E7EE12D0A330780302C36A307B30E530540FF582
:20C4000058906000E054F04558F0E558B40700401A906020E054F04558F0E558B40A0C9079
:20C420006040742AF0906060743AF0906000E0540FF558F530B40400500512B5A3802BB465
:20C4400004054321038023B4050543210C801BB4060575210F8013B40705432103800BB4A3
:20C46000080543210C800375210F90CFFAE55893C4F559F5501278AC7F00FEAD837B0A121D
:20C48000AD9F8559501278B87F00FEAD837B2012AD9FE558B404004065B404187F007E5083
:20C4A0007D617B0A12AD9F7F007EA07D607B2012AD9F804AB405187F007E707D617B0A12CB
:20C4C000AD9F7F007EE07D607B2012AD9F802FB4062F7F007E507D617B0A12AD9F7F007EBA
:20C4E000A07D607B2012AD9F7F407E607D617B2012AD9F7F807EC07D607B4012AD9F02C558
:20C5000097B407187F107E507D617B0A12AD9F7F207EA07D607B2012AD9F807BB408187FB2
:20C52000107E707D617B0A12AD9F7F207EE07D607B2012AD9F8060B409447F007E507D615D
:20C540007B0A12AD9F7F107E607D617B0A12AD9F7F107E707D617B0A12AD9F7F007EA07D72
:20C56000607B2012AD9F7F207EC07D607B2012AD9F7F207EE07D607B2012AD9F8019B40A85
:20C58000167F107E507D617B3012AD9F7F207EA07D607B6012AD9F123C0C75D018302EFD5C
:20C5A000C23075A08090FF927B027440123B062275D018E530540FF55812CE9212CFC450A4
:20C5C00006432FC002D10B90D1A01273C378C97447F6906190E4F0A3740DF012AEABD23034
:20C5E000E55EF55A540C03F55C03C4906F90F0F5501278C5F552E55CFF90BDF893CF049356
:20C60000F5828F83E55D541823C493F5557553F0E4F554F55BF55C85525D85535E85545FF7
:20C6200012D085E55AF30925F0F5F0E55BF30925F0F5F0E55CF30925F0F5F07F4090E008BA
:20C64000E552F0855383855482E0A3858254E583700474F00552F55390E004E0A3FEE0C3A8
:20C660001392D5F30925F0F5F0A2D5EE13C313F30925F0F5F0E555B55204D27C8002DFBD55
:20C6800012D0F875D018E500B501101264F2302BF5127A0250F0D27A02D10B12D00540E3FE
:20C6A000B44318207C2AE55B3401A2E7C2E7F55BE55A3400C2E7F55A02C617B44E0C855D74
:20C6C00052855E53855F5402C620B44FB602D12A12D0BD75D018E500B5010F1264F2302B93
:20C6E000F5127A0250F0D27A80AE12D00540E4B44302800BB44E0280D7B44FD702D12A75C7
:20C70000D018E500B501101264F2302BF5127A0250F0D27A02D10B12D00540E3B441028055
:20C7200006B44FDB02D12A12D041B401E712D04170E212D04170DD12D04170D812D041B432
:20C74000030050D0F55F12D041B44A0050C6F55E12D0412401255F255EC2E770B712D04196
:20C7600030E7B1E55FC313F55FF55DE55E92E7F55EF55C12D0857401F309F5F0E4F309E450
:20C78000F309906F90E0F5501278ACF5517F09E0A3F30925F0F5F0155EE55EB4FF04E55FBB
:20C7A000155FDFEB906F90E0F5501278B8F5527F20E0A3FE540FF30925F0F5F0155EE55ECF
:20C7C000B4FF02155FEEC4540FF30925F0F5F0155EE55EB4FF06E55F6015155FDFD37583DF
:20C7E00061E5512410F5827F09E55F455E700302C83DE0A3F30925F0F5F0155EE55EB4FF2C
:20C8000002155FDFED758360E5522420F5827F20E0A3FE540FF30925F0F5F0155EE55EB4A9
:20C82000FF02155FEEC4540FF30925F0F5F0155EE55EB4FF06E55F6004155FDFD312D0F861
:20C8400075D018E500B501101264F2302BF5127A0250F0D27A02D10B12D00540E3B443021D
:20C860008012B44E09855D5F855C5E02C773B44FCF02D12AE55F455E700302C91512D085EF
:20C880007401F309E4F3097452F30975F0539061607F09E0A3F30925F0F5F0DFF69060C0F6
:20C8A0007F20E0A3FE540FF30925F0F5F0EEC4540FF30925F0F5F0DFE99061707F09E0A3C0
:20C8C000F30925F0F5F0DFF69060E07F20E0A3FE540FF30925F0F5F0EEC4540FF30925F01E
:20C8E000F5F0DFE912D0F875D018E500B501101264F2302BF5127A0250F0D27A02D10B12E7
:20C90000D00540E3B44302800CB44E0302C87DB44FD502D12A12D0BD75D018E500B50110D2
:20C920001264F2302BF5127A0250F0D27A02D10B12D00540E3B44302800BB44E0280D6B4AB
:20C940004FD602D12A75D018E500B501101264F2302BF5127A0250F0D27A02D10B12D00516
:20C9600040E3B441028006B44FDB02D12A12D041B401E712D041B408E112D04170DC12D06C
:20C980004170D712D04170D212D041B428CC12D0412431C2E770C312D04130E7BD12D0852D
:20C9A0007401F3097408F309E4F30975F0099064007F14E0A3FE540FF30925F0F5F0EEC42D
:20C9C000540FF30925F0F5F0DFE912D0F875D018E500B501101264F2302BF5127A0250F0CE
:20C9E000D27A02D10B12D00540E3B44302800CB44E0302C99DB44FD502D12A12D0BD75D058
:20CA000018E500B501101264F2302BF5127A0250F0D27A02D10B12D00540E3B4431675D047
:20CA200018302EFDC23075A08090FF927B027440123B0622B44E0280DAB44FC202D12A75A0
:20CA4000D01812CE9290D1B01273C378C97447F69061907401F0A3740DF012AEABD230E5E5
:20CA60005EF55A540C0303C4F5501278C5F55212D0A37553F0E4F554F556F55BF55C75D069
:20CA800018E500B501101264F2302BF5127A0250F0D27A02D10B12D00540E3B44202800F92
:20CAA000B44F0302D12AB445D512D0A302CB7AE556C2E7255CA2E7C2E7F55CE556548023BF
:20CAC000355BA2E7C2E7F55BE55A3400C2E7F55A75F00012D041B55ABA25F0F5F012D0416B
:20CAE000B55BB025F0F5F012D041B55CA625F0F5F075560085525D85535E85545F90E008C3
:20CB0000E552F0855383855482F0A3858254E583700474F00552F55312D041FE12D0412007
:20CB2000E72005560556C5F025F0C5F0233392D590E004F0A3EEC5F025F0C5F0A2D533F0EE
:20CB400080BBE5F02EC2E7701DE554C39401F554E553540F940044F0F553E5529400F552CA
:20CB600012D0A302CA7E12D0DE855D52855E53855F54755600C27C02CA7E75D018E500B53A
:20CB800001101264F2302BF5127A0250F0D27A02D10B12D00540E3B440028006B44FDB026E
:20CBA000D12A12D041B401E7F5F012D04170E012D04170DB12D04170D612D041B403005062
:20CBC000CEF55F25F0F5F012D041B44A0050C0F55E25F0F5F012D04125F0C2E770B112D0D7
:20CBE0004130E7ABE55FC313F55FF55DE55E92E7F55EF55C12D0A375D018E500B501101273
:20CC000064F2302BF5127A0250F0D27A02D10B12D00540E3B44202800FB44F0302D12AB42E
:20CC200045D512D0A302CDB812D041B401DE12D04170D912D04170D475F0019061007F0966
:20CC400012D041F0A325F0F5F0155EE55EB4FF04E55F155FDFEA9060007F2012D041FE2561
:20CC6000F0F5F0155EE55EB4FF02155F12D041C5F025F0C5F0C44EF0A3155EE55EB4FF064A
:20CC8000E55F600F155FDFD39061107F09E55F455E700302CCDE12D041F0A325F0F5F01567
:20CCA0005EE55EB4FF04E55F155FDFEA9060207F2012D041FE25F0F5F0155EE55EB4FF0266
:20CCC000155F12D041C5F025F0C5F0C44EF0A3155EE55EB4FF06E55F6004155FDFD312D07A
:20CCE00041FE12D04130E707EE25F0C2E7600C12D0DE855D5F855C5E02CBF712D0A375D0CE
:20CD000018E500B501101264F2302BF5127A0250F0D27A02D10B12D00540E3B44202800F0F
:20CD2000B44F0302D12AB445D512D0A302CDB812D041B401DE12D04170D912D041B452D3F8
:20CD400075F0539061207F0912D041F0A325F0F5F0DFF59060407F2012D041FE25F0F5F014
:20CD600012D041C5F025F0C5F0C44EF0A3DFE99061307F0912D041F0A325F0F5F0DFF590E7
:20CD800060607F2012D041FE25F0F5F012D041C5F025F0C5F0C44EF0A3DFE912D041FE12D7
:20CDA000D04130E707EE25F0C2E7600612D0DE02CCFE12D0A302CCFE75D018E500B501104D
:20CDC0001264F2302BF5127A0250F0D27A02D10B12D00540E3B440028006B44FDB02D12A42
:20CDE00012D041B401E712D041B408E112D04170DC12D04170D712D04170D212D041B42877
:20CE0000CC12D0412431C2E770C312D04130E7BD12D0A375D018E500B501101264F2302BAB
:20CE2000F5127A0250F0D27A02D10B12D00540E3B44202800FB44F0302D12AB445D512D0C1
:20CE4000A302C3F812D041B401DE12D041B408D812D04170D375F0099064007F1412D04187
:20CE6000FE25F0F5F012D041C5F025F0C5F0C44EF0A3DFE912D04125F0C2E7600912D0413E
:20CE800012D0DE02CE1312D04130E7F412D0A302CE13207817906F8074F0F0A37441F0A3EC
:20CEA000E531F0A37410F0A37412F022906F0074F0F0A37441F0A3E531F0A37410F0A374A8
:20CEC00040F0906F1074F0F0A37441F0A3E531F0A37410F0A37441F0906F2074F0F0A374E5
:20CEE00041F0A3E531F0A37410F0A37442F0906F3074F0F0A37441F0A3E531F0A37410F06D
:20CF0000A37443F0A374F7F0906F4074F0F0A37441F0A3E531F0A37410F0A37445F0A374CB
:20CF2000F7F0906F5074F0F0A37441F0A3E531F0A37410F0A3744EF0A374F7F0906F607439
:20CF4000F0F0A37441F0A3E531F0A37410F0A3744FF0A374F7F02290CFFAE55893F55912EA
:20CF6000B5AF6050E559C4F5501278B8F551E0540FB55845B405004039E5590412B5AF60EF
:20CF800033E5512420758360F582E0540FB55829B406028005B409004018300A179060C045
:20CFA000E0540FB55813300B0B9060E0E0540FB55807C32290B603800390B6231273C3122D
:20CFC00078F6D322E55E540C0303F55912B5AF601EE55DB405004015E5590412B5AF600F8C
:20CFE000E55DB409004006300A05300B02C32290B6031273C31278F6D3220001020300027D
:20D00000000002000075D0007568658568A012D04120E706E8B501F6D322B4F0F712D04183
:20D02000B441F112D041B531EB12D041B410E512D041FAB44300400612D04130E7D6EAC333
:20D040002275D000E8B5010280FAE208222078012275D0087568668568A0906F007F05E008
:20D06000A3F309DFFA75F000222078012275D0087568668568A0906F107F05E0A3F309DFE8
:20D08000FA75F0002275D0087568668568A0906F20207803906F807F05E0A3F309DFFA7568
:20D0A000F000222078012275D0087568668568A0906F307F06E0A3F309DFFA801820780149
:20D0C0002275D0087568668568A0906F407F06E0A3F309DFFA302EFDD29975D01822207818
:20D0E000012275D0087568668568A0906F507F06E0A3F309DFFA80DDE5F0F404C2E7F309F5
:20D1000074F7A3F309302E02D29922207E0330781975D0087568668568A0906F607F06E0D5
:20D12000A3F309DFFA302EFDD299C23075D018207F1790D1D01273C31278F6207A0B126498
:20D14000F2302BFA127A0250F5302EFD53A8C175D01875A08090FF927B027440123B0622E5
:20D1600053616D706C65204461746120586D742053616D706C65204461746120586D742ABB
:20D1800053616D706C652044617461205263762053616D706C652044617461205263762AB7
:20D1A000586D742053616D706C652044617461205263762053616D706C6520446174612093
:20D1C000205761697420666F7220446174612020202020202043616E63656C2020202020D3
:20D1E00075D01853A8819000311273C31264F2302BFA90D22C1273C31278F6906000E0B5B5
:20D200008215A3E583B470F6E478FFF690D23C1273C31278F6804574FFF8F612DC1490D211
:20D220004C1273C31264F2302BFA803020436865636B204261636B20757020204261636BA8
:20D24000207570204E6F204572726F72204261636B207570204572726F72202090D2F4125A
:20D2600073C31278F6906000E4F0A3E583B470F8906000755F00E0B55F65A3E583B470F6CB
:20D2800090600074FFF0A3E583B470F7906000755FFFE0B55F49A3E583B470F6906000748C
:20D2A00055F0A3E583B470F7906000755F55E0B55F2DA3E583B470F690600074AAF0A3E51E
:20D2C00083B470F7906000755FAAE0B55F11A3E583B470F690D3041273C31278F6804574B0
:20D2E000FFF8F612DC1490D3141273C31264F2302BFA8030436865636B20526561642F5713
:20D30000726974652020522F57204E6F204572726F722020526561642F57726974652045DF
:20D3200072726F7290D49A1273C3755A0090D4CAE55A2323FF93F551EF04FF93F550EF04CB
:20D34000FF93F553EF0493F552755B10755CF0755D0090E008E55BF0855C83855D82F090C3
:20D36000E004E550F0A3E551F0855C83855D82A3F085835C85825D90E004E552F0A3E55342
:20D38000F0E55D2401F55DE4355CF55C70CA755CF0055B1264F2302B0B7875E644E7B4E75C
:20D3A0000302D429E55BB430A9755B10755CF0755D0090E008E55BF0855C83855D82E0904B
:20D3C000E004E054F0B55061A3E0B5515C855C83855D82A3E085835C85825D90E004E0543F
:20D3E000F0B55245A3E0B55340E55D2401F55DE4355CF55C70C2755CF0055B1264F2302B91
:20D400000A7875E644E7B4E702801EE55BB430A2E55A04F55AB40202800302D32D90D4AA26
:20D420001273C31278F602D4DA74FFF8F612DC14755F04E55BB420005003755F0790E00483
:20D44000E55D20E018E054F0B55028A3155FE0540FF8E551540FB5181A155F8016E054F021
:20D46000B55210A3155FE0540FF8E553540FB51802155F90D4BA1273C375A08078007482FC
:20D48000F2087431F208E55F2430F208123AFB1278ED1264F2302BFA8040202020436865B6
:20D4A000636B204452414D20202020204452414D204E6F204572726F722049432020202063
:20D4C0004452414D204572726F725550AAA0AAA0555055505550AAA0AAA0126D0090D64914
:20D4E0001273C3752F0090680074F0F0A374E7F0A374E0F0A374F0F0A374E0F0A374E0F05A
:20D50000A374ECF0A31264F2302BFA7480F5A07800F2087F087420F208DFFC1278ED74C022
:20D520007800F2087F087420F208DFFC1278ED78C0E6FF906800E04FF0EF540F60087F00A5
:20D540001340320F80FA78C1E6FF906801E04FF0EF541860097F0520E4027F04801778C2E5
:20D56000E6FF906802E04FF0EF541F60137F061340030F80FA8F30123C0CEF12ADFD8074BC
:20D5800078C3E6FF906803E04FF0EF540F60087F001340520F80FA78C4E6FF906804E04F9E
:20D5A000F0EF541F60087F0413403B0F80FA78C5E6FF906805E04FF0EF541F60087F091374
:20D5C00040240F80FA78C6E6FF906806E04FF0EF5413604F7F0E1340030F80FAEFB41206F2
:20D5E00090C000747FF0EF23FF90D65993CF0493F5828F837480F5A07800F2087F03742095
:20D60000F208DFFCC3123AE0B809121278ED780074C0F208C3123AE0B809028003123AFBDA
:20D620001278ED7875E644E7B4E70974FFF8F612DC14800C7F07906800E0A3B4FF08DFF94E
:20D640001278F602D70002D50520506C65617365205075736820537720D67FD685D68AD66B
:20D6600093D699D69ED6A3D6AAD6B1D6B7D6BCD6C6D6D2D6DED6E3D6EBD6F4D6F4D6F520A4
:20D68000205245430D4D4F44450D5354414E445F42590D53544152540D4C4F41440D534174
:20D6A00056450D4631202F203E0D4632202F203C0D454E5445520D54554E450D5041524169
:20D6C0004D455445520D57415645204D4F444946590D504552464F524D414E43450D4D49C3
:20D6E00044490D464F52574152440D4241434B574152440D0D415250204F4E2F4F46460D5E
:20D7000090D7731273C3752F0078C97445F6906191740DF07B4153A8DDC230906190EBF07E
:20D7200012AEAB753C00D23043A8A21278D3E53C20E716B41000401AEB04B45B0050E4B49F
:20D74000410040DFFBD27880CDB4F1005004EB1480E81264F2302BD37875E644E7B4E7093F
:20D7600074FFF8F612DC1480033078BF53A8DDC23080102020414C504841204449414C2002
:20D7800020202090D8341273C3755000795FE55090B000F01278D3E0C2E0F7190550B95BEB
:20D7A000ED752F00755000795FE55090B000F01278D3E754F0FFE0C2E0FE54F0B51F028035
:20D7C0000CAF500FE4D333DFFD452FF52FEEF7190550B95BD475A08078007485F208795FBE
:20D7E000E719FF12DC21EEF208EFF208123AFB1278ED780074C0F208E719FF12DC21EEF2F8
:20D8000008EFF2A3B95B261278D31264F2302B947875E644E7B4E70974FFF8F612DC148009
:20D8200023E52F540FB40F02801A02D7A4087420F20880C4414443202020202020202020B0
:20D840002020202090D90B1273C3E4F510F511F52FFF906700F0A3DFFC90517F7409F090B8
:20D86000517CE090517DE090517F7408F043A888E510B511201264F2302BF57875E644E7ED
:20D88000B4E70974FFF8F612DC1480033078E153A8F702D92B758367851082E0A320E70974
:20D8A000E582B511F6F51080C7C2E724DDFEE0A3858210C2E7FD20780890D91B1273C3D2D3
:20D8C000787568808568A078007484F208E51E75F00A842430F208E5F02430F208123AFBCE
:20D8E0001278ED780074C4F208E51D75F064842430F208E5F075F00A842430F208E5F0245B
:20D9000030F208123AFB1278ED809C506C656173652050757368204B6579204B6579202017
:20D9200020202056656C202020202090D9621273C31278F6E4126ECB20080A74FFF8F61259
:20D94000DC1402DABB906083E004F090D9721273C31264F2302BFA78C4E630E1F4126EB3BF
:20D960008020436865636B2051442053797374656D20506C656173652050757368205341E1
:20D98000564575A08090B8067B017440123B0675510075520190DA6B1273C3E4F521906FE2
:20D9A00000F012B32D05510552E552B404E753A8DD755A0090DA5FE55A23FF93CF0493F543
:20D9C000828F831273C3E4FE7F4012896AE55A75F002A42404C4FF74017E0012896A740222
:20D9E0007E007F0012896AE55A0375F004A42404FE740412896A74057EFF7F7F12896AE555
:20DA00005A90DA6793FF7EFF740612896A90E0007401F074137EFF7F3F12896A1264F23019
:20DA20002BFA7875E644E7F4601BF4B4E7EE74FFF8F612DC1474137E007F0012896A90E07B
:20DA400000E4F0807674137E007F0012896A90E000E4F0055AE55AB40402805F02D9B4DA8F
:20DA60007BDA8BDA9BDAAB7FFF7FFF434F50592020202020202020202020202020436865C5
:20DA8000636B2042414E4B203120202020436865636B2042414E4B203220202020436865AF
:20DAA000636B2042414E4B203320202020436865636B2042414E4B2034202090DBA4127347
:20DAC000C31278F690DBB41273C31264F2302BFA90DBA41273C31278F65398E053A8C1750C
:20DAE000D0087568668568A0E4F8F9F500F50190DB7EE493A36004F30980F7439812D2AC79
:20DB000075D0187F007E101264F2202B43E501B509028006DFF1DEEF801B5398E053A8C1BA
:20DB2000A80075A06590DB7EE493A3601AFFE208B51F0280F390DBC41273C31264F2302BDA
:20DB4000FA74FFF8F6800990DBD41273C31278F690DBE41273C31278F612DC1478FFE66004
:20DB60000890DBF41273C380FE90DC041273C31264F2302BFA7874E620E4F402004153554E
:20DB80005A554B49204753582D5220202034303055484F4E44412020494E54454752412094
:20DBA00047534900202020436865636B204D494449202020436F6E6E65637420494E2D4FA4
:20DBC000555420214D4944492048617264204572726F722020204D494449204E6F20457238
:20DBE000726F7220456E64206F6620436865636B20507267506C6561736520506F776572D8
:20DC0000204F6666506C65617365205075736820456E7472906000E582F0A3E583B470F789
:20DC200022EFC4540FB40A0050052430FE80032437FEEF540FB40A0050042430FF22243737
:20DC4000FF22C0E0C0D075D00075A065E599F309E500B50104D252D25E753B148568A0D026
:20DC6000D0D0E0C29832C0E0C0D075D00875A066E8B50904D22E8006E2F59908C22E85681B
:20DC8000A0D0D0D0E032C0E0C0D0C083C08275D01090517CE02424F57890517DE0F5797545
:20DCA000A067E578F309E579F309E510B51102D25F8568A0D082D083D0D0D0E032C0E0C0A8
:20DCC000D0C0F08878C3E534703275340AB257E53860021538E53960021539E53A6002155A
:20DCE0003AE53B6002153B788EE6600116E53D6002153D305706E53E6002153EE53420E061
:20DD00002E7883E6C423F5F0441F2536F536E5F0541F3535F5355002B227301812201A0F95
:20DD2000E53F6004153F80077880E6F53FD219202C0AE53D7004D22C8002153D153420302C
:20DD40000302DDAE8979C083C08278C779C806B6000107E710E729B6F019B70016D2D50925
:20DD6000E7F9540FC990619012DDBF79C8E792E7F78032B6682FB7012CE4F6F7C2D580DF26
:20DD8000F778C9E6540F906190A304B408FB78C779C8B6F107B70004D2D58002C2D57440C6
:20DDA000790012DDBFA979D082D0838568A0758CF6758A3CD28CA878D0F0D0D0D0E032F501
:20DDC0007A448075A0807800F208E0A3B40D097480F208B809FBC32230D5027420F2080984
:20DDE000B908E7B80909E57A5440C37001D3227480F20880EEC0E0C0D020911730960B056B
:20DE00003CE53CB4800D153C8009153CE53CB47F02053CC2CED0D0D0E03200000000000090
:20DE20000000000000000000000000000000000000000000000000000000000000000000E2
:20DE40000000000000000000000000000000000000000000000000000000000000000000C2
:20DE60000000000000000000000000000000000000000000000000000000000000000000A2
:20DE8000000000000000000000000000000000000000000000000000000000000000000082
:20F30000C60102030405060708FFFFFEF3EBE5E0DCD9D5D3D2CFCECDCBCBCAC9C8C7C8C685
:20F32000C6C6C5C5C5C4C4C4C3C4C3C3C3C3C2C2C2C2C2C1C1C2C1C1C1C1C1C13BC13DC185
:20F340003F404142434445464748494A4A4C4D4D4F505052525454565658585A5A5C5C5CE8
:20F360005F5F6161616464646767676A6A6A6D6D6D6D7171717175757575757A7A7A7A7EE6
:20F38000C50102030405060708FFFAF0E8E1DCD9D5D2D1CECDCCCACAC8C8C7C7C7C6C6C673
:20F3A000C5C5C4C4C3C3C2C2C3C2C2C2C1C2C1C1C1C1C132C13435363738393A3B3C3D3D7B
:20F3C0003F40414143434545474749494B4B4D4D4D505050535353565656565A5A5A5A5A7C
:20F3E0005F5F5F5F5F6464646464646A6A6A6A6A6A70707070707076767676767676767E90
:20F40000003300360038003C004000440048004C00510055005B00600066006C00720079D9
:20F4200000800087008F009800A100AA00B500BF00CB00D700E400F10100010F011F013006
:20F4400001420155016A017F019601AE01C801E30200021E023E0260028502AB02D402FF66
:20F46000032C035D039003C60400043C047D04C1050A055605A805FE065906BA0720078D23
:20F480000800087908FA09830A140AAD0B500BFC0CB20D740E410F1A100010F311F5130635
:20F4A0001428155B16A017F919651AE81C821E34200021E723EB260D28512AB72D412FF218
:20F4C00032CB35D139043C68400043CE47D64C1C50A3556E5A825FE465986BA3720978D1CE
:20F4E0008000879C8FAD9838A145AADCB505BFC9CB30D745E412F1A2FFFFFFFFFFFFFFFF17
:20F500000030003300360039003D004100440048004D00510056005B00610066006C00731A
:20F52000007A008100890091009900A300AC00B600C100CD00D900E600F40102011101229F
:20F54000013301450158016D0183019A01B201CC01E70204022302430266028A02B102DAF0
:20F56000030503330364039803CE04080446048704CB0514056205B4060B066606C8072F10
:20F58000079C0810088B090D09970A290AC40B670C150CCD0D900E5E0F3910211116121A25
:20F5A000132E1452158716CF182A199A1B201CBD1E722041222C2435265C28A42B0E2D9E30
:20F5C00030543334363F39793CE44083445948694CB85147561D5B3B60A866686C7E72F21F
:20F5E00079C8810688B290D2996FA28FAC39B677C150CCCFD8FD008000800080008000805B
:20F600000000000100020003000400050006000700080009000A0D000D010D020D030D0468
:20F620000D050D060D070D080D090D0A0E000E010E020E030E040E050E060E070E080E0996
:20F640000E0A081008200830085008800821083108510881083208420872084308730854D6
:20F660000884087508870910092009300950098009010921093109510981090209120932E2
:20F6800009420972090309130923094309730924093409540984090509150945097509270C
:20F6A00009370957098709080918094809780A100A200A300A500A800A010A210A310A51E8
:20F6C0000A810A020A120A320A420A720A030A130A230A430A730A240A340A540A840A05EB
:20F6E0000A150A450A750A270A370A570A870A080A180A480A7800000001000200030004A7
:20F7000001010101020203030404050506060707080809090A0A0B0B0C0C0D0D0E0E0F0FF7
:20F72000101010101111111112121212131313131414141415151515161616161717171759
:20F74000181818181818181819191919191919191A1A1A1A1A1A1A1A1B1B1B1B1B1B1B1B79
:20F760001C1C1C1C1C1C1C1C1D1D1D1D1D1D1D1D1E1E1E1E1E1E1E1E1F1F1F1F1F1F1F1FD9
:20F78000202020202020202020202020202020202121212121212121212121212121212159
:20F7A0002222222222222222222222222222222223232323232323232323232323232323F9
:20F7C000242424242424242424242424242424242525252525252525252525252525252599
:20F7E000262626262626262626262626262626262727272727272727272727272727272739
:20F8000027283034383A3C3E4041424344454647484849494A4A4B4B4C4C4D4D4E4E4F4F75
:20F82000505050505151515152525252535353535454545455555555565656565757575758
:20F84000585858585858585859595959595959595A5A5A5A5A5A5A5A5B5B5B5B5B5B5B5B78
:20F860005C5C5C5C5C5C5C5C5D5D5D5D5D5D5D5D5E5E5E5E5E5E5E5E5F5F5F5F5F5F5F5FD8
:20F88000606060606060606060606060606060606161616161616161616161616161616158
:20F8A0006262626262626262626262626262626263636363636363636363636363636363F8
:20F8C000646464646464646464646464646464646565656565656565656565656565656598
:20F8E000666666666666666666666666666666666767676767676767676767676767676738
:20F90000000202030405060708090B0C0D0E0F10111214151617191A1C1D1E1F21222324BC
:20F920002627292A2C2D2F303233353637383A3B3D3E404143444647494A4B4D5153555730
:20F94000595B5D5E60626466686A6C6E70727577797B7D7F828486888A8C8F919395979A9F
:20F960009C9FA2A4A7AAADB0B3B6B9BBBEC1C4C7CBCED2D6D9DCDFE2E5E9EEF2F6F9FDFF21
:20F98000FFFBF7F3EFEBE7E3DFDBD7D3CFCBC7C3C0BDBAB7B4B1AEABA8A5A29F9C999693BF
:20F9A000908E8C8A88868482807E7C7A78767472706E6C6A68666462605E5C5A5856545227
:20F9C000504E4C4A48464442403E3C3A38363432302F2D2C2B2A292827262524232221209D
:20F9E0001F1E1D1C1B1A191817161514131211100F0E0D0C0B0A0908070706060505040407
:20FA0000FFFBF7F3EFEBE7E3DFDBD7D3CFCBC7C3C0BDBAB7B4B1AEABA8A5A29F9C9996933E
:20FA2000908E8C8A88868482807E7C7A78767472706E6C6A68666462605E5C5A58565452A6
:20FA4000504E4C4A48464442403E3C3A38363432302F2D2C2B2A292827262524232221201C
:20FA60001F1E1D1C1B1A191817161514131211100F0E0D0C0B0A0908070605040302020194
:20FA80000080008000008000800080000102040810204080FEFDFBF7EFDFBF7F202020206E
:20FAA00020202020200D2020200D204F4E4F46463153484F54204D414E204155544F20416F
:20FAC00055544F32465744414C5442574420555020444F574E552F4420524E44206F63740E
:20FAE00054524947474154454649582056454C4F494E5420455854204D494449424F544806
:20FB000048414C46434F4E544348524D2043200D4323200D2044200D4423200D2045200D92
:20FB20002046200D4623200D2047200D4723200D2041200D4123200D2042200D202D200D49
:20FB400020412020422020432020442041422043442041424344412F42432F4441422F43EA
:20FB600044412F422F432F44456D7074794475564D56534454444C4D53542054554E4520FE
:20FB80003D202020200D4D494449204348414E4E454C3D0D4D4944492042454E4445523DE5
:20FBA0000D4D49444920484F4C4420203D0D4D494449204D4F442020203D0D50474D204330
:20FBC00048414E4745203D0D4143542053454E53494E473D0D5245472D504152414D202043
:20FBE0003D0D4558434C555349564520203D0D564942205241544520203D0D4D2D56494267
:20FC000020445054483D0D442D56494220445054483D0D442D56494220444C41593D0D4137
:20FC20005250205241544520203D0D415250204D4F444520203D0D4152502052414E47452A
:20FC4000203D206F63740D415250205245504541543D0D415250204445434159203D0D549F
:20FC6000524720472D54494D453D0D5452472D20207E202020202D0D562D53572054485211
:20FC800053483D0D562D4D582054485253483D0D44454C41592054494D453D0D44454C4146
:20FCA00059204C45564C3D0D232020203D0D205B202020202020205D207E0D4152502053C8
:20FCC000594E4320203D0D4454554E204D4F4445203D0D4454554E2052414E47453D0D4272
:20FCE000454E442044455354203D0D42454E44204D4F4445203D0D4142454E442044455355
:20FD0000543D0D50495443482042454E443D0D5649425241544F2020203D0D4544543A0D65
:20FD200053504C543A0D524543204B45592020203D0D42414E4B2054554E453D2020202077
:20FD40000D4C4F4F5020545950453D0D5343414E204D4F4445203D0D5354203D0D454E44F4
:20FD60003D0D4C50203D0D4B455920464F4C4C4F573D0D44594E2053454E5345203D0D42D8
:20FD8000454E4420524E473D2020205B20205D41454E3D0D414C503D0D4C4F4F50205455A8
:20FDA0004E453D202020200D4B4559204F46465345543D0D454E5620562D53454E533D0DBD
:20FDC000454E56205241544531203D0D454E56204C4556454C313D0D454E56205241544522
:20FDE00032203D0D454E56204C4556454C323D0D454E56205241544533203D0D454E56208F
:20FE00004C4556454C333D0D454E56205241544534203D0D44594E2053454E5345203D0D27
:20FE20004142454E4420524154453D0D4142454E4420445054483D0D2020526F6C616E643E
:20FE400020532D3130202020436F6E6669726D696E67204C6F6164204E6F726D616C205399
:20FE6000617665204D6F646550666D20446174612050726F74656374204661737420536161
:20FE80007665204D6F6465204475616C20546F6E65202056656C6F2D4D697820202056653A
:20FEA0006C6F2D5377697463682020446574756E65202020202044656C61792020202020F4
:20FEC000577269746520436F6D706C65746520202020202052656164790D20202052414DBC
:20FEE000204552524F52212020204564697474696E670D20457874204761746520506C6163
:20FF0000790D20204275666665722046756C6C21212020204D656D6F727920496E6974201F
:20FF20002020506572666F726D616E636520496E69742020204D49444920496E69742020E4
:20FF40002020204D73742054756E6520496E6974202020436F707920436F6D706C65746549
:20FF60002020532E53747263743D20202020202020202041737369676E204D6F64652D30EC
:20FF800020204D6F64652D3120204D6F64652D3220201F11111111111F001F151B151B15B3
:20FFA0001F001F1F1F1F1F1F1F00040E1F1F040E1F1F00000000040E1F1F1F1F0E04040EF7
:20FFC0001F1F1F1F0E04000000001F1F0E041F1F0E040E04000000001F1F0E041F1F0E0441
:20FFE000000000000000000000000000000000000000000000000000000000000000000001
:00000001FF
